:100000000C9439020C9456020C9456020C9456022D
:100010000C9456020C9456020C9456020C94560200
:100020000C9456020C94DC0C0C9456020C94560260
:100030000C9406160C9456020C9456020C9456021C
:100040000C9456020C9456020C94B70B0C94560266
:100050000C94F5040C9456020C94BF040C945602B4
:100060000C94880D0C9456020C9460150C94560256
:100070000A0A0D004E65757472616C004865616412
:10008000696E67486F6C64000A0D5374657565721C
:10009000756E673A20004F4B0A0D000A0D416267EA
:1000A0006C65696368204C756674647275636B7304
:1000B000656E736F722E2E000A0D42656E75747A2E
:1000C0006520506172616D657465727361747A2028
:1000D0002564000A0D414343206E69636874206102
:1000E000626765676C696368656E21000A0D496E19
:1000F00069742E20454550524F4D3A2047656E6534
:1001000072696572652044656661756C742D506115
:1001100072616D657465722E2E2E000A0D3D3D3D97
:100120003D3D3D3D3D3D3D3D3D3D3D3D3D3D3D3DFF
:100130003D3D3D3D3D3D3D3D3D3D3D000A0D466C57
:1001400069676874436F6E74726F6C0A0D486172F0
:1001500064776172653A25642E25640A0D536F66D3
:1001600074776172653A5625642E256425632044B0
:1001700061726B4D6F64205625642E2564002E003D
:1001800048693A253469202043663A2534692000BD
:1001900047733A253469202047693A25346920009D
:1001A0004E693A2534692020526F3A25346920007F
:1001B00045787465726E436F6E74726F6C202000A8
:1001C00052616E67653A2533692D25336900537492
:1001D000656C6C756E673A202533690053657470E1
:1001E0006F696E74202025336900536572766F2025
:1001F0002000506F7469343A202025336900506F15
:100200007469333A202025336900506F7469323A9B
:10021000202025336900506F7469313A202025333E
:10022000690053746172743A2020202020253569BA
:10023000004D657373776572743A20202535690027
:100240005269636874756E673A2020253569004BE2
:100250006F6D706173732020202020202000456D79
:1002600070662E506567656C3A253569005370617C
:100270006E6E756E673A202025356900486F636899
:100280002025346920282533692900526F6C6C20A1
:10029000253469202825336929004E69636B2025A0
:1002A000346920282533692900414343202D2053F8
:1002B000656E736F72004769657220253469202866
:1002C0002533692900526F6C6C202534692028255C
:1002D000336929004E69636B202534692028253352
:1002E000692900476965722025346920282533690A
:1002F0002900526F6C6C2025346920282533692928
:10030000004E69636B202534692028253369290054
:100310004779726F202D2053656E736F72005033D2
:100320003A253469202050343A2534692000503170
:100330003A253469202050323A2534692000477329
:100340003A253469202047693A25346920004E69EE
:100350003A2534692020526F3A25346920004B3702
:100360003A25346920204B383A25346920004B3532
:100370003A25346920204B363A25346920004B3326
:100380003A25346920204B343A25346920004B311A
:100390003A25346920204B323A25346920004B6FCE
:1003A0006D706173733A20202025356900526F6C9F
:1003B0006C3A202020202020253569004E69636B8F
:1003C0003A20202020202025356900616B742E20E2
:1003D0004C6167650048F668656E726567656C75A7
:1003E0006E67004B65696E6520004F6666202020B1
:1003F0002020203A20253569004C7566746472759A
:10040000636B3A2025356900536F6C6C486F6568E3
:10041000653A2025356900486F6568653A202020D7
:1004200020202535690028632920486F6C67657294
:1004300020427573730053657474696E673A2025A2
:1004400064200048573A5625642E25642053573AB5
:1004500025642E25642563002B204D696B726F4B3C
:100460006F70746572202B005B25695D005B2569E8
:100470005D0011241FBECFEFD0E1DEBFCDBF13E082
:10048000A0E0B1E0EEE1FBE702C005900D92A43AD6
:10049000B107D9F717E0A4EAB3E001C01D92AE3D61
:1004A000B107E1F70E94B2020C948D3D0C9400005C
:1004B0009C01F999FECF32BD21BDF89A80B508950F
:1004C0009C01F999FECF1FBA32BD21BD60BD0FB6A8
:1004D000F894FA9AF99A0FBE0895F999FECF22E09E
:1004E00030E032BD21BDF89A80B5863060F0F999D0
:1004F000FECF1FBA32BD21BD82E080BD0FB6F89499
:10050000FA9AF99A0FBE08951F93182F863008F0B3
:1005100015E0419FC001112420E632E050E08C59E3
:100520009F4F0E94903AF999FECF1FBA82E090E067
:1005300092BD81BD10BD0FB6F894FA9AF99A0FBE1C
:100540001F910895FB01863008F085E0489FB001B7
:1005500011246C597F4F28E532E050E0CF010E9412
:10056000743A08958F929F92AF92BF92CF92DF928A
:10057000EF92FF920F931F93CF93DF9314B815B8A8
:10058000189B02C08BE001C08AE0809300018DE8D7
:1005900087B98FEF88B98BE184B981E085B98EE3A3
:1005A0008AB9579A87EF8BB984B7877F84BF8091C8
:1005B00060008861809360001092600080ED97E099
:1005C0009093C6038093C50310925C0410925B0461
:1005D00010921A071092190710925A041092590497
:1005E0001092580410925704809100018A3011F43F
:1005F000289801C0289A42980E94700C0E94CB064D
:100600000E94F1150E94820D0E942215789410928A
:100610000C0684E480930D0687E080930E062091FB
:10062000000181E090E09F938F931F921F9284E6D8
:1006300090E09F938F9384E490E09F938F931F9219
:100640001F92822F6AE00E94E63C892F90E09F93E0
:100650008F93822F0E94E63C90E09F938F938CE3D0
:1006600091E09F938F931F920E94FA088BE191E093
:100670009F938F931F920E94FA08299A8DB79EB775
:1006800044960FB6F8949EBF0FBE8DBFF999FECF6A
:10069000C1E0D0E0D2BDC1BDF89A80B5853409F47F
:1006A0003BC08CEE90E09F938F931F920E94FA08BC
:1006B0000E94AC3910E00F900F900F90123039F07B
:1006C000133019F40E948A3804C0143010F00E94CC
:1006D0001B3947E461E477E0812F0E9484021F5FA9
:1006E000163061F7F999FECF1FBA82E090E092BD13
:1006F00081BD83E080BD0FB6F894FA9AF99A0FBED7
:10070000F999FECF1FBAD2BDC1BD85E480BD0FB639
:10071000F894FA9AF99A0FBEF999FECF84E090E026
:1007200092BD81BDF89A80B5853050F083ED90E0A0
:100730009F938F931F920E94FA080F900F900F9033
:100740000E946D0247E461E477E00E94A2020E94E9
:100750006D0290E09F938F9388EB90E09F938F932F
:100760001F920E94FA08809149070F900F900F90F6
:100770000F900F9080FD03C0C8EED3E020C08BE93E
:1007800090E09F938F931F920E94FA0888EE93E067
:100790000E94970CEC010E941C100F900F900F907C
:1007A000CE010E94A10C8823D9F386E990E09F93A3
:1007B0008F931F920E94FA080F900F900F900E9443
:1007C0006621809100018A3011F4289801C0289A8E
:1007D00080ED97E09093C6038093C50385E58093F1
:1007E000160688E890E09F938F931F920E94FA0864
:1007F000809149070F900F900F9082FF03C08CE704
:1008000090E002C084E790E09F938F931F920E9434
:10081000FA080F900F900F9080E790E09F938F93CE
:100820001F920E94FA080E94751088E893E1909345
:100830008703809386030F900F900F9030E7832EED
:1008400037E1932EA12C23E0B22E95E0C92ED12CB6
:1008500080E1E82E87E2F82E00E810E08091C203E4
:100860008823E1F31092C2030E94EC220E9424210B
:10087000809100018A3011F4289801C0289A809153
:100880000301882321F081508093030112C010924C
:10089000B4031092B50310922006109279041092BE
:1008A000780410927B0410927A0410927D041092C6
:1008B0007C0480915604882329F08091560481504D
:1008C000809356048091860390918703892BD1F4FD
:1008D000D0928703C09286030E9431158091040351
:1008E000909105038F5F9F4FE9F480915F04882307
:1008F000C9F0F092C603E092C5031093050300937C
:10090000040310C080918603909187030197909310
:10091000870380938603809100018A3011F4289820
:1009200001C0289A8091C203882311F40E94E60630
:100930000E948E07CE010E94A10C882309F48ECF5D
:100940002091090330910A038091590790E02817FC
:1009500039077CF480910403909105038F5F9F4FCA
:1009600041F49092C6038092C503B0920503A09211
:10097000040384E690E00E94970CEC016FCF1F9275
:100980000F920FB60F9211248F939F93EF93FF93C3
:10099000809101018823E1F48091BE039091BF030F
:1009A00001969093BF038093BE03FC01E252FB4F7C
:1009B000E081ED3019F08639910539F41092BF03CA
:1009C0001092BE0381E080930101E093C60004C051
:1009D0001092BF031092BE03FF91EF919F918F91F0
:1009E0000F900FBE0F901F9018951F920F920FB689
:1009F0000F9211242F933F934F938F939F93AF9315
:100A0000BF93CF93DF93EF93FF938091C6008093C2
:100A1000A8034091B903463910F01092B8038091B1
:100A2000A8038D3009F05CC08091B803823009F0D2
:100A300057C01092B803A42FB0E0FD01E15EF94F5A
:100A40003081ED01C05ED94F28818091BC03909127
:100A5000BD03831B9109821B91099F709093BD0375
:100A60008093BC039C0196E0369527959A95E1F713
:100A7000235C2093BB03982F9F73935C9093BA03DE
:100A80008081281729F48881981711F491E006C015
:100A90008091AB038F5F8093AB0390E08091A903BB
:100AA000882309F069C0992309F466C081E0809326
:100AB000A9034093AC03AF5DB94F8DE08C93809157
:100AC0002306823509F058C02CE088E190E00FB68B
:100AD000F894A895809360000FBE209360004CC0EE
:100AE0008091B8038130F9F0813020F0823009F034
:100AF00041C024C08091A803833239F48091A903B6
:100B0000882319F481E08093B8038091A80380932F
:100B1000210681E08093B9038091A8038093BC03F0
:100B20001092BD0329C082E08093B803E42FF0E067
:100B30008091A803EF5DF94F808309C0E42FF0E0B6
:100B40008091A803EF5DF94F8083463920F44F5F11
:100B50004093B90302C01092B8032091A80380917A
:100B6000BC039091BD03820F911D9093BD038093B0
:100B7000BC0302C01092B803FF91EF91DF91CF91B7
:100B8000BF91AF919F918F914F913F912F910F9076
:100B90000FBE0F901F901895DC0120E030E040E080
:100BA00050E008C0FA01E252FB4F8081280F311D4E
:100BB0004F5F5F4F4A175B07A8F33F70C90136E0EC
:100BC000969587953A95E1F7835CFD01E252FB4FDC
:100BD000808311962F73235CFD01E252FB4F20832B
:100BE000A152BB4F8DE08C93109201018091DE04E5
:100BF0008093C6000895CF93DF93EA01B22F93E26A
:100C00009093DE046093DF048093E00463E070E07F
:100C1000A0E04EC0FE01EA0FF11D9081AF5FB15020
:100C200019F430E040E00FC0FE01EA0FF11D4081F1
:100C3000AF5FB15011F430E006C0FE01EA0FF11DC4
:100C40003081AF5FB150892F86958695835CFB011B
:100C5000E252FB4F8083242F22952F70892F90E042
:100C60008370907054E0880F991F5A95E1F7282BF4
:100C7000235CFB01E152FB4F2083842F90E08F70B7
:100C80009070880F991F880F991F232F2295269502
:100C900026952370282B235CFB01E052FB4F208319
:100CA0003F73335CFB01EF51FB4F30836C5F7F4F31
:100CB000BB2309F0AFCFCB010E94CC05DF91CF91D0
:100CC00008951F93CF93DF93EC0170E0A22FB0E063
:100CD000119748C0E42FF0E0EF5DF94F30814F5F8E
:100CE000E42FF0E0EF5DF94F50814F5FE42FF0E02B
:100CF000EF5DF94F10814F5FE42FF0E0EF5DF94FAA
:100D000020814F5F842F90E08A179B0774F55D5315
:100D1000FE01E70FF11D852F82958F703D53330F34
:100D2000330F382B3083613001F1912F9D537F5F5A
:100D3000FE01E70FF11D71505295507F892F869566
:100D40008695582B5083623081F063507E5FFE01A0
:100D5000E70FF11D9295990F990F907C2D53922BCF
:100D600090837F5F662309F0B5CFDF91CF911F910C
:100D700008951F93182F8A3019F48DE00E94B90648
:100D80008091C00085FFFCCF1093C60080E090E00A
:100D90001F9108950895E1ECF0E088E18083A0ECD4
:100DA000B0E08C9182608C938081806880838081A8
:100DB000806480838AE28093C40088EC90E00E9483
:100DC000970C90930B0680930A0608958091010179
:100DD000882309F4A2C08091A403882371F0809134
:100DE0000101882351F02BE046E156E06091DD04DB
:100DF00087E40E94FB051092A40380910A0690915B
:100E00000B060E94A10C882321F48091A60388235D
:100E1000B1F080910101882391F022E447EB56E084
:100E20006091DD0484E40E94FB051092A60384EF28
:100E300091E00E94970C90930B0680930A066091B4
:100E400002016F3F89F0462F50E074E0440F551FB8
:100E50007A95E1F74C5F5E4F605D20E181E40E948E
:100E6000FB058FEF809302019091F9069923A1F081
:100E700080910101882381F083E28093DE049093C6
:100E8000DF048DE08093E004109201011092F906D6
:100E90008091DE048093C6008091A503882359F1D8
:100EA00080910101882339F10E947E101092A503E0
:100EB0003091AE03932F9F5F9093AE03943021F057
:100EC0008091AF03882359F026E145E157E060E0C7
:100ED00084E30E94FB058FEF8093AE030CC044E1D6
:100EE000949FA0011124455E5C4F24E160E0832FB4
:100EF0008F5C0E94FB058091A703882371F080918D
:100F00000101882351F02AE04CE056E06091DD04B5
:100F100086E50E94FB051092A70308951F93DF93B7
:100F2000CF9300D0CDB7DEB78091A903882309F411
:100F300006C18FEF80930301809123068B3609F45D
:100F400079C08C3688F48336D1F1843630F481361A
:100F5000C1F0823609F0F1C020C0873609F47BC0A9
:100F6000883609F0EAC042C0813709F478C0813779
:100F700008F49DC0843709F454C0863709F0DDC0F9
:100F800066C02091AC0343E062E0CE0101960E946E
:100F90006106898180930201D0C02091AC0343E0B7
:100FA0006BE086E196E00E9461068091ED039091EE
:100FB0001806892B8093ED0380911F0645C0209170
:100FC000AC0343E06BE086E196E00E94610680910D
:100FD000ED0390911806892B8093ED0380911F06F5
:100FE0008093F90681E08093A603A7C02091AC030B
:100FF00043E062E0CE0101960E9461068091ED031C
:101000009981892B8093ED038A818F3F21F481E0C0
:101010008093AF0302C01092AF0381E08093A503D9
:101020008CC02091AC0343E064E080EB93E00E942D
:10103000610683C02091AC0343E064E084EB93E05D
:101040000E9461068091B7038093F90676C081E023
:101050008093A70372C081E08093A4036EC02091A7
:10106000AC0343E062E0CE0101960E9461068981F3
:101070008F3F89F0863010F085E0898347E461E492
:1010800077E089810E94A202898127E441E457E048
:101090006091DD0408C01091DD040E946D0227E418
:1010A00041E457E0612F855B0E94FB0546C020911B
:1010B000AC0343E067E481E497E00E94610680911D
:1010C000230647E461E477E08B560E948402209176
:1010D0002306F999FECF1FBA82E090E092BD81BD50
:1010E0002B5620BD0FB6F894FA9AF99A0FBE60916C
:1010F0006C0770E080E090E024EC39E040E050E0E4
:101100000E94C73C609388037093890380938A038D
:1011100090938B0360916D0770E080E090E00E94F7
:10112000C73C60938C0370938D0380938E039093E0
:101130008F030E946D020E94D2221092A9030F9089
:101140000F90CF91DF911F910895982F8091FA060B
:10115000813061F48091EC03E82FF0E0E55EFC4F14
:1011600090838F5F8093EC0381E00895892F0E9424
:10117000B90608951F93182F04C080E30E94A508A4
:1011800011501116D4F31F9108951F93182F04C006
:1011900080E20E94A50811501116D4F31F91089502
:1011A0000F931F93CF93DF938C01EB0108C0F801DD
:1011B0000F5F1F4FE4918E2F0E94A5082197209763
:1011C000B1F7DF91CF911F910F9108950F931F9366
:1011D000CF93DF938C01EB0106C0F80181918F0161
:1011E0000E94A50821972097C1F7DF91CF911F9109
:1011F0000F9108952F923F924F925F926F927F923C
:101200008F929F92AF92BF92CF92DF92EF92FF9216
:101210000F931F93DF93CF93CDB7DEB7E5970FB64C
:10122000F894DEBF0FBECDBF2C969FAD2C972D96A8
:101230004FAD2D972B968FAD2B978093FA06FDE43B
:10124000AF2EB12CAC0EBD1E292F342FC9019DA786
:101250008CA71EA61FA618AA19AA9E01245D3F4F9F
:101260003DAB2CAB0CA51DA502C00F5F1F4FF801B5
:10127000F490FF2019F0F5E2FF16B9F7B8012CA59C
:101280003DA5621B730B19F0C9010E94D008FF2015
:1012900009F454C2A8014F5F5F4F5DA74CA71982A4
:1012A00044241BAA5FEF5AAB02C0C5015C01ECA548
:1012B000FDA5CF0101969DA78CA76491A42DB0E058
:1012C000A170B070653721F0862F80628837F1F405
:1012D000109771F0F50120813181428153812EA751
:1012E0003FA748AB59AB24E030E0A20EB31E0EC0BE
:1012F000F501808191819C0140E050E02EA73FA73D
:1013000048AB59AB42E050E0A40EB51E603221F468
:101310008981882351F61AC0633211F458E05AC00B
:101320006A3221F06D3281F4C50109C0C50102960F
:10133000D501BC91BBABB7FFB9CFB195BBABE0E179
:101340004E2AFFED4F22B2CF6B3211F46983ADCF3D
:101350006E3209F03AC0ECA5FDA59F012F5F3F4F0B
:101360003DA72CA784918A3221F0682F20E030E03D
:1013700021C0C5010296D5014D915C9157FF02C075
:101380004FEF5FEF4AAB92CFC901E3E0880F991F9F
:10139000EA95E1F7220F331F280F391F260F311D61
:1013A00020533040ECA5FDA5AF014F5F5F4F5DA717
:1013B0004CA76491862F80538A3030F3A90137FF00
:1013C00002C04FEF5FEF4AAB7DCF603329F444FC9E
:1013D0006CCF50E2452A69CF862F81538930E8F4DB
:1013E00020E030E0C90153E0880F991F5A95E1F7DA
:1013F000220F331F280F391F260F311D2053304075
:10140000ECA5FDA5CF0101969DA78CA76491862F21
:1014100080538A3038F32BAB55CF683619F494E0FB
:10142000492A43CF6C3619F4A1E04A2A3ECF562E02
:10143000F501B3E66B1741F422E030E0A20EB31ED3
:1014400080818C83198227C134E4631739F044E624
:10145000641731F059E66517C1F502C081E0482AEA
:1014600040FE09C0A4E0B0E0AA0EBB1E208131817D
:10147000428153810BC042E050E0A40EB51E808132
:1014800091819C01442737FD4095542F2EA73FA7FB
:1014900048AB59AB8EA59FA5A8A9B9A9B7FF11C0A4
:1014A0002EA53FA548A959A950954095309521955D
:1014B0003F4F4F4F5F4F2EA73FA748AB59AB3DE281
:1014C0003983562E0AE0302E82C04FE4641721F093
:1014D0005FE6651731F402C081E0482A18E0312E3A
:1014E00075C090E76917A1F4A2E0B0E0AA0EBB1E98
:1014F000808191819C0140E050E02EA73FA748AB3E
:1015000059AB30E4432AB0E13B2EA8E75A2E5EC027
:101510006337E1F5D501CD90DC90C114D10489F495
:10152000B8E2BC83EEE6ED83F5E7FE832CE62F837D
:10153000288739E239871A86F4E0CF2ED12CCC0ED9
:10154000DD1E4AA947FD10C0552747FD509560E0B4
:1015500070E0C6010E94673A009771F0182F1C19BD
:101560005AA951174CF009C0F60101900020E9F783
:1015700031971E2F1C1901C01AA982E090E0A80E15
:10158000B91E1982E3E75E2E40E08CC0653521F07C
:10159000653739F4562E02C091E0492A7AE0372E99
:1015A00015C0683519F0683709F06FC043FE0BC0ED
:1015B0002EA53FA548A959A9211531054105510579
:1015C00011F030E4432A562E60E1362E19824AA9E2
:1015D00047FD02C05FED45228EA59FA5A8A9B9A928
:1015E0000097A105B10549F49AA9992331F45CE269
:1015F000C52ED12CCC0EDD1E44C0EEA4FFA408A93C
:1016000019A94CE2C42ED12CCC0EDD1E632C7724FC
:1016100088249924C801B701A40193010E94193DAF
:101620006A3020F430E3232E260E08C027E5222E50
:10163000260EA8E55A1611F4BFED2B22F6012292D0
:101640006F01C801B701A40193010E94193DC901AE
:10165000DA018EA79FA7A8ABB9ABE614F70408057B
:10166000190518F07C018D01D5CFF8E03F1649F43B
:1016700043FE07C020E3221621F0D601E0E3EE93FB
:101680006D011CA91C194AA90DC0662309F456C096
:101690006C831982562E40E011E094E0C92ED12CC3
:1016A000CC0EDD1E042F011B07FD00E0898188237D
:1016B00019F0812F8F5F06C046FC02C0812F02C047
:1016C000812F8E5F782E700EE42CFF2480E3882E0D
:1016D000912C8E209F208114910421F48BA98719CD
:1016E0000E94C5088981882329F061E070E0CE015D
:1016F000019609C0E6FE09C0F0E3FA835B8262E06E
:1017000070E0CE0102960E94E60820E28216910463
:1017100021F48BA987190E94BA08802F0E94BA0869
:10172000612F772767FD7095C6010E94E608E4FEE9
:1017300099CD8BA987190E94C50894CDE5960FB65F
:10174000F894DEBF0FBECDBFCF91DF911F910F91F7
:10175000FF90EF90DF90CF90BF90AF909F908F90D1
:101760007F906F905F904F903F902F9008951F92C1
:101770000F920FB60F9211242F933F935F936F93A5
:101780007F938F939F93AF93BF938091C9038150B1
:101790008093C9038F5FB9F489E08093C903809176
:1017A00008038F5F817080930803882319F481E018
:1017B0008093C2038091C0039091C10301969093DE
:1017C000C1038093C0038091C5039091C603029723
:1017D000E8F08091C5039091C60301979093C603EA
:1017E0008093C5038091C5039091C60320910403A3
:1017F0003091050382239323892B31F0429A809103
:101800000603882371F415C0429813C0429881E002
:10181000809306038FEF9FEF90930503809304035B
:1018200008C0809100018A3011F45A9A09C0479A81
:1018300007C0809100018A3011F45A9801C047987E
:101840008091490783FF3BC0349B0AC08091C3034A
:101850009091C40301969093C4038093C3032FC057
:101860008091C3039091C403892B79F08091C303C5
:101870009091C403805A9F4040F48091C30390919B
:10188000C40390934704809346048091460490914A
:1018900047042091480430914904845E9D4F821B87
:1018A000930B68E671E00E94063D845B9040909344
:1018B0004B0480934A041092C4031092C303BF9157
:1018C000AF919F918F917F916F915F913F912F91F8
:1018D0000F900FBE0F901F901895809306030895E8
:1018E0008091C0039091C1030B969093CB0380939A
:1018F000CA0382E085BD83EA84BD17BC88E788BD42
:1019000096E096BD83EC8093B0009093B100E0E741
:10191000F0E0808182608083EEE6F0E0808181608B
:1019200080838AE08093B3001092B20008952091E2
:10193000C0033091C1032F5F3F4F280F391FC901EA
:1019400008952091C0033091C103821B930B8070D6
:101950009078892F869508952091C0033091C10316
:101960002F5F3F4F280F391F8091C0039091C10313
:10197000A901481B590BCA0180709078892F869560
:1019800099F308952091C0033091C1032F5F3F4F19
:10199000280F391F4FEE02C040937A008091C00398
:1019A0009091C103B901681B790BCB0180709078CD
:1019B000892F869589F308951F920F920FB60F9283
:1019C00011242F933F934F935F936F937F938F9344
:1019D0009F93AF93BF93CF93DF93EF93FF93809148
:1019E00007038150809307038F5F09F074C083E879
:1019F0008093B00080919D03C82FD0E0D093C8039E
:101A0000C093C7038091760780FF1EC060910A04CF
:101A100070910B0480910C0490910D0420E830E04B
:101A200040E050E00E943B3DCA01B90120916307AC
:101A300030E040E050E00E94C73C20E032E040E06F
:101A400050E00E943B3D24C060910A0470910B0459
:101A500080910C0490910D0420E830E040E050E0CB
:101A60000E943B3DCA01B9012091630730E040E08C
:101A700050E00E94C73C20E032E040E050E00E948D
:101A80003B3D50954095309521953F4F4F4F5F4FCF
:101A9000C20FD31FD093C803C093C7032091C703BD
:101AA0003091C8038091640790E02817390734F01B
:101AB0008091650790E08217930724F49093C80300
:101AC0008093C7038091C7038093B300809166071A
:101AD0008093070304C083E08093B0005F98FF9178
:101AE000EF91DF91CF91BF91AF919F918F917F91B6
:101AF0006F915F914F913F912F910F900FBE0F907B
:101B00001F90189510927C008FEE80937A000895B4
:101B10001F920F920FB60F921124EF92FF920F9324
:101B20001F932F933F934F935F936F937F938F9365
:101B30009F93AF93BF93EF93FF9310927A0080919E
:101B4000E8038F5F8093E8038150853009F486C0F5
:101B5000863090F4823009F440C0833030F488231A
:101B6000F1F0813009F044C22FC0833009F441C044
:101B7000843009F03DC25AC0883009F4C2C08930AF
:101B800038F4863009F483C0873009F031C29CC034
:101B9000893009F4D3C08A3009F02AC2AFC18091DC
:101BA0007800909179009093E7038093E60381E0B9
:101BB0008093E9038091E0039091E1030196909373
:101BC000E1038093E00318C280917800909179003E
:101BD0009093E5038093E40392C080917800909104
:101BE00079009093E3038093E20384E08093E90318
:101BF00003C24091090350910A03809178009091AB
:101C000079009A01220F331F240F351F63E070E023
:101C10000E94F23C260F371F36952795369527955B
:101C200030930A032093090386E0E0CF80910204F9
:101C3000909103042091780030917900821B930BDE
:101C40009093FC068093FB068091FB069091FC0626
:101C50009093D3038093D20387E0C8CF809178001C
:101C6000909179002091000430910104821B930B24
:101C700090930707809306078091060790910707C6
:101C80009093D5038093D4031092E903B5C180915A
:101C900000012091E6033091E7038A3049F48091F6
:101CA000780090917900820F931F9695879506C0D2
:101CB0008091780090917900820F931F9093D103C7
:101CC0008093D00381E092CF809100012091E403C2
:101CD0003091E5038A3049F4809178009091790041
:101CE000820F931F9695879506C0809178009091FA
:101CF0007900820F931F9093CF038093CE0382E0ED
:101D000075CF809100012091E2033091E3038A3086
:101D100049F48091780090917900820F931F9695F5
:101D2000879506C08091780090917900820F931F6B
:101D30009093CD038093CC0385E058CF60917800D9
:101D400070917900E0900404F0900504009106047D
:101D500010910704882777FD8095982F0E94B03B4B
:101D6000A80197010E94AC3A0E947D3B7093D70373
:101D70006093D6034091D6035091D7038091FB0620
:101D80009091FC06209106073091070797FF03C04A
:101D9000909581959F4F959587959595879537FF58
:101DA00003C0309521953F4F35952795359527955B
:101DB000820F931F840F951F9093D7038093D603B0
:101DC0008091D6039091D703029704F160910404A7
:101DD00070910504809106049091070420E030E0A2
:101DE00048E454E40E94113B88230CF03CC060910D
:101DF00004047091050480910604909107042AE080
:101E000037ED43EA5CE30E94AD3A25C08091D603EA
:101E10009091D7038F5F9F4F34F5609104047091C8
:101E20000504809106049091070420E030E046E12B
:101E300054E40E94603C1816B4F46091040470915C
:101E4000050480910604909107042AE037ED43EAE7
:101E50005CE30E94AC3A60930404709305048093A1
:101E600006049093070481E08093DD03809178005D
:101E7000909179009093FE068093FD062091420494
:101E80003091430440914404509145048091D6031D
:101E90009091D703AA2797FDA095BA2F820F931F81
:101EA000A41FB51F8093420490934304A09344045D
:101EB000B0934504E0904204F09043040091440440
:101EC0001091450460914204709143048091440450
:101ED0009091450420E034E040E050E00E943B3D1A
:101EE000E21AF30A040B150BE0924204F092430449
:101EF000009344041093450483E078CE80910B074F
:101F000090910C072091780030917900820F931FF7
:101F100090930C0780930B07809103078F5F80934A
:101F2000030780910307853008F462C08091780030
:101F3000909179009093100380930F031092030700
:101F40008091FF069091000720910B0730910C07BC
:101F5000821B930B2091600430916104821B930BD0
:101F60009093DF038093DE0320910B0730910C07E1
:101F7000E0900B03F0900C0300910D0310910E0301
:101F8000C801B701660F771F881F991F6E0D7F1D4F
:101F9000801F911F442737FD4095542F620F731FF8
:101FA000841F951F24E030E040E050E00E943B3D5C
:101FB000C901DA0180930B0390930C03A0930D03E6
:101FC000B0930E032091FF063091000780910B0320
:101FD00090910C03A0910D03B0910E03281B390BB7
:101FE000309361042093600410920C0710920B0749
:101FF0001092E9031092E8038091E90380937C003A
:102000008091E803882319F08FEE80937A00FF9186
:10201000EF91BF91AF919F918F917F916F915F9160
:102020004F913F912F911F910F91FF90EF900F9043
:102030000FBE0F901F901895EF92FF920F931F9372
:10204000CF93DF93F999FECF03E0E02E00E0F02E6E
:10205000F2BCE1BCF89A80B5C82FD0E0C531D105FB
:1020600008F02A97C7BD84E690E00E94C20C8091D8
:102070000F039091100382559340C8F4C0E0D0E064
:1020800016C0C7BD82E390E00E94C20C1F930F935D
:102090001F920E94FA0880910F03909110030F90F5
:1020A0000F900F908458934038F0219602C00EE7AD
:1020B00011E0CA3FD10528F38C2FF999FECF1FBA42
:1020C000F2BCE1BC80BD0FB6F894FA9AF99A0FBE43
:1020D000809308078CE291E00E94C20CDF91CF91BF
:1020E0001F910F91FF90EF900895EBE1F3E080E2F4
:1020F000819393E0EB36F907D9F70895FF920F9398
:102100001F938091ED03282F30E080FF15C0809150
:10211000EE03882311F0815002C080916B038093FD
:10212000EE03EBE1F3E080E2819393E0EB36F90715
:10213000D9F78FEF8093AE0321FF10C08091EE039B
:102140008F5F8093EE03EBE1F3E080E2819393E015
:10215000EB36F907D9F78FEF8093AE032370307019
:102160002330310511F41092EE038091EE03282FF5
:1021700030E08A3040F481E18093EC033F932F9369
:102180008DE694E007C080E18093EC033F932F93AA
:1021900088E694E09F938F9381E08F930E94FA08E2
:1021A0000F900F900F900F900F901091EE0315303D
:1021B00009F403C2163090F4123009F4D0C0133081
:1021C00030F4112309F1113009F031C465C0133026
:1021D00009F41BC1143009F02AC46BC1183009F48A
:1021E00021C3193038F4163009F4A1C2173009F0B0
:1021F0001EC4F4C21A3009F48FC31A3008F450C355
:102200001B3009F014C4C6C31092EC0388E594E0B7
:102210009F938F9311E01F930E94FA0884E18093AB
:10222000EC032091000184E690E09F938F9384E477
:1022300090E09F938F931F921F92822F6AE00E94DB
:10224000E63C892F90E09F938F93822F0E94E63C7B
:1022500090E09F938F9383E494E09F938F931F93D9
:102260000E94FA0888E28093EC030E946D0290E0DD
:102270009F938F9386E394E09F938F931F930E9485
:10228000FA088CE38093EC0386E294E09F938F93AB
:102290001F930E94FA089EC28091490780FF47C0A1
:1022A0001092EC0380916004909161049F938F934E
:1022B00087E194E09F938F931F930E94FA0884E133
:1022C0008093EC0380916204909163049F938F93B9
:1022D00088E094E09F938F931F930E94FA0888E20E
:1022E0008093EC0380910F03909110039F938F9341
:1022F00089EF93E09F938F931F930E94FA088CE3DA
:102300008093EC038091080790E09F938F938AEE6F
:1023100093E09F938F931F930E94FA088DB79EB707
:1023200044960FB6F8949EBF0FBE8DBF85C384E15F
:102330008093EC0383EE93E09F938F931F930E940F
:10234000FA0888E28093EC0385ED93E09F938F93E6
:102350001F930E94FA088DB79EB70696E2CF10929F
:10236000EC038BEC93E09F938F9311E01F930E94FB
:10237000FA0884E18093EC0360910A0470910B04E5
:1023800080910C0490910D0420E034E040E050E096
:102390000E943B3D5F934F933F932F938CEB93E0D1
:1023A0009F938F931F930E94FA0888E28093EC0317
:1023B000609112047091130480911404909115049B
:1023C00020E034E040E050E00E943B3D5F934F93BB
:1023D0003F932F938DEA93E09F938F931F930E94D7
:1023E000FA088CE38093EC038091460490914704B3
:1023F0009F938F938EE993E09F938F931F930E94F7
:10240000FA088DB79EB746968CCF1092EC03809158
:10241000190790911A0720911707309118079F9379
:102420008F933F932F938EE893E09F938F9311E0C8
:102430001F930E94FA0884E18093EC0380911D07AA
:1024400090911E0720911B0730911C079F938F933B
:102450003F932F938EE793E09F938F931F930E9458
:10246000FA0888E28093EC0380912107909122077B
:1024700020911F07309120079F938F933F932F93B5
:102480008EE693E09F938F931F930E94FA088CE34C
:102490008093EC03809125079091260720912307D4
:1024A000309124079F938F933F932F938EE593E072
:1024B0007BC01092EC03E0914207F0E0EE0FFF1FAB
:1024C000EB5EF84F20813181E0914107F0E0EE0FA3
:1024D000FF1FEB5EF84F808191813F932F939F9375
:1024E0008F938EE493E09F938F9311E01F930E944C
:1024F000FA0884E18093EC03E0914407F0E0EE0FEA
:10250000FF1FEB5EF84F20813181E0914307F0E03F
:10251000EE0FFF1FEB5EF84F808191813F932F9369
:102520009F938F938EE393E09F938F931F930E94CB
:10253000FA0888E28093EC03E0914607F0E0EE0FA2
:10254000FF1FEB5EF84F20813181E0914507F0E0FD
:10255000EE0FFF1FEB5EF84F808191813F932F9329
:102560009F938F938EE293E09F938F931F930E948C
:10257000FA088CE38093EC03E0914807F0E0EE0F5B
:10258000FF1FEB5EF84F20813181E0914707F0E0BB
:10259000EE0FFF1FEB5EF84F808191813F932F93E9
:1025A0009F938F938EE193E09F938F931F930E944D
:1025B000FA088DB79EB74C96B4CE1092EC0380E12A
:1025C00093E09F938F9311E01F930E94FA080F905E
:1025D0000F900F90809100018A3009F052C084E181
:1025E0008093EC034091F6035091F7038091CC0364
:1025F0009091CD032091F6033091F7035F934F93B1
:10260000821B930B9F938F9381E093E09F938F9313
:102610001F930E94FA0888E28093EC034091F8032C
:102620005091F9038091CE039091CF032091F8034C
:102630003091F9035F934F93821B930B9F938F937A
:1026400082EF92E09F938F931F930E94FA088CE38E
:102650008093EC038091FA039091FB032091B007E3
:102660003091B1079F938F933F932F9383EE92E026
:102670009F938F931F930E94FA088DB79EB745963C
:1026800050CE84E18093EC038091F6039091F703A0
:102690002091CC033091CD03E091F603F091F70344
:1026A00062E070E00E94063D7F936F932E1B3F0B0C
:1026B0003F932F9384ED92E09F938F931F930E94FB
:1026C000FA0888E28093EC038091F8039091F90373
:1026D0002091CE033091CF03E091F803F091F903FC
:1026E00062E070E00E94063D7F936F932E1B3F0BCC
:1026F0003F932F9385EC92E09F938F931F930E94BB
:10270000FA088CE38093EC038091FA039091FB0329
:102710002091B0073091B10762E070E00E94063D61
:102720007F936F933F932F9386EB92E0A1CF10920C
:10273000EC0389EA92E09F938F93FF24F394FF9236
:102740000E94FA0884E18093EC0380910004909148
:1027500001042091D4033091D5039F938F933F932D
:102760002F938AE992E09F938F93FF920E94FA0839
:1027700088E28093EC0380910204909103042091FD
:10278000D2033091D3039F938F933F932F938BE882
:1027900092E09F938F93FF920E94FA088CE38093BC
:1027A000EC036091040470910504809106049091FB
:1027B000070400919807109199070E947D3B7F9331
:1027C0006F931F930F938CE792E09F938F93FF92E9
:1027D0000E94FA088DB79EB74896A3CD84E18093F6
:1027E000EC038091090390910A039F938F938DE6E8
:1027F00092E09F938F9311E01F930E94FA0888E262
:102800008093EC038091560490E09F938F938EE524
:1028100092E09F938F931F930E94FA088DB79EB703
:102820000A967FCD1092EC038FE492E09F938F93F2
:1028300011E01F930E94FA0884E18093EC038091D9
:102840004A0490914B049F938F9380E492E09F936E
:102850008F931F930E94FA0888E28093EC03809183
:102860004604909147049F938F9381E392E09F9356
:102870008F931F930E94FA088CE38093EC0380915E
:102880004804909149049F938F9382E292E09F9332
:102890008F931F930E94FA088DB79EB7429641CD41
:1028A0001092EC0380914E0490914F049F938F936C
:1028B00086E192E09F938F9311E01F930E94FA08A4
:1028C00084E18093EC0380915004909151049F9394
:1028D0008F938AE092E09F938F931F930E94FA0850
:1028E00088E28093EC0380915204909153049F936B
:1028F0008F938EEF91E09F938F931F930E94FA081E
:102900008CE38093EC0380915404909155049F9341
:102910008F9382EF91E0FDCC1092EC038AEE91E070
:102920009F938F9311E01F930E94FA0884E1809394
:10293000EC0380919D0390E09F938F938CED91E049
:102940009F938F931F930E94FA0888E28093EC0371
:102950008091C7039091C8039F938F938EEC91E071
:102960009F938F931F930E94FA088CE38093EC034C
:102970008091650790E09F938F938091640790E02A
:102980009F938F9380EC91E09F938F931F930E946E
:10299000FA08C4CC1092EC0380EB91E09F938F93E4
:1029A00011E01F930E94FA0884E18093EC03809168
:1029B0001A06992787FD90959F938F93809119060A
:1029C000992787FD90959F938F9380EA91E09F933D
:1029D0008F931F930E94FA0888E28093EC03809102
:1029E0001B06992787FD90959F938F9380911C06D6
:1029F00090E09F938F9380E991E09F938F931F9333
:102A00000E94FA088CE38093EC038091200690E00A
:102A10009F938F9380911D06992787FD90959F9393
:102A20008F9380E891E09F938F931F93D1CE1150A5
:102A300010936B031092EE031092ED031F910F9110
:102A4000FF9008951092B9008AE28093B80008952B
:102A500085EA8093BC0080E0089584E98093BC00FF
:102A600008954CEB50E084E9DA018C931092EF0367
:102A70002BEB30E0F90180811092F00380E88C9319
:102A80001092BD001092BA001082E9EBF0E01082C3
:102A9000A8EBB0E01C9210828AE28C9385EADA01FE
:102AA0008C931082F901108285E88C93089510921E
:102AB000B9008093BB0085E88093BC0080E0089556
:102AC0001F920F920FB60F9211248F939F93EF9343
:102AD000FF938091EF038F5F8093EF0381508330EA
:102AE00061F1843038F48130A9F09091F0038230A4
:102AF000C0F40AC0853031F1853060F1863051F183
:102B0000873009F060C044C0892F90E08996880F13
:102B1000991F33C08091F0038F5F8093F003815041
:102B20001BC084E98093BC00943018F41092EF032A
:102B300002C01092F00385EA25C08091F103880F4E
:102B40008D5A1BC08091BB00E091F103F0E0E35F80
:102B5000F84F80838091F103813051F0813028F06B
:102B6000823049F0833079F510C080918B0705C021
:102B70008091900702C08091A8071092B9008093BD
:102B8000BB0085E88093BC001EC08091AA07F5CFEA
:102B90008091F1039091BB00E82FF0E0E35FF84FE4
:102BA00094838F5F8093F103843010F01092F103CF
:102BB00084E98093BC008AE090E09093870380933F
:102BC00086031092EF038091BC0080688093BC0064
:102BD000FF91EF919F918F910F900FBE0F901F90DB
:102BE000189583EC80938100EFE6F0E080818062AD
:102BF00080831092FB031092FA031092F903109253
:102C0000F8031092F7031092F60308951F920F92A3
:102C10000FB60F9211240F931F932F933F934F934F
:102C20005F936F937F938F939F93AF93BF93CF9354
:102C3000DF93EF93FF93209186003091870080917E
:102C4000F4039091F503281B390B80918600909135
:102C500087009093F5038093F403C9018D54944049
:102C60000091F2031091F303835F9A4160F4043002
:102C7000110514F010926C0381E090E09093F3033F
:102C80008093F2038AC00A3011050CF086C0C90196
:102C90008B5F9040845B914008F068C0E901C25DA1
:102CA000D140F801EE0FFF1FEB5EF84F808191815C
:102CB0009E01281B390BC90137FF03C090958195F0
:102CC0009F4F06974CF480915604883C28F48091DD
:102CD0005604865F80935604F801EE0FFF1FEB5EEB
:102CE000F84F20813181C901880F991F820F931FEE
:102CF0008C0F9D1F64E070E00E94063D9B01CE0199
:102D00000196861797071CF42150304006C0219782
:102D10006C177D0714F42F5F3F4F80915604E80134
:102D2000CC0FDD1F833CB8F0FE01EB5EF84F8081D5
:102D30009181A901481B590BCA0163E070E00E9410
:102D4000063DCB01880F991F860F971FC55DD84F91
:102D50009983888304C0C55DD84F19821882F80111
:102D6000EE0FFF1FEB5EF84F31832083F8013196A1
:102D7000F093F303E093F203E530F10511F45D9A6B
:102D800006C05D98E630F10511F45C9A05C05C98C8
:102D9000379711F45B9A01C05B98FF91EF91DF9137
:102DA000CF91BF91AF919F918F917F916F915F91E3
:102DB0004F913F912F911F910F910F900FBE0F9048
:102DC0001F9018952F923F924F925F926F927F9231
:102DD0008F929F92AF92BF92CF92DF92EF92FF922B
:102DE0000F931F93DF93CF9300D0CDB7DEB78091C1
:102DF000FA039091FB032091D0033091D103821B01
:102E0000930B9093B1078093B0078091CE0390917C
:102E1000CF032091F8033091F903821B930B909319
:102E20008A07809389078091CC039091CD032091EC
:102E3000F6033091F703821B930B909392078093D4
:102E400091078091890790918A079093F206809369
:102E5000F106E090AD07F090AE076091D403709159
:102E6000D503882777FD8095982F2CE030E040E04F
:102E700050E00E94C73C0027F7FC0095102FE60E9B
:102E8000F71E081F191FC801B70122E030E040E01B
:102E900050E00E943B3D3093AE072093AD07E09099
:102EA000B707F090B8076091D2037091D3038827D9
:102EB00077FD8095982F2CE030E040E050E00E94B4
:102EC000C73C0027F7FC0095102FE60EF71E081FE1
:102ED000191FC801B70122E030E040E050E00E9435
:102EE0003B3D3093B8072093B70720919807309166
:102EF00099076091D6037091D703882777FD809555
:102F0000982F442737FD4095542F620F731F841F5D
:102F1000951F22E030E040E050E00E943B3D3093BE
:102F200099072093980740911A0450911B046091CF
:102F30001C0470911D042091D4033091D503C90164
:102F4000880F991F820F931F880F991F880F991F51
:102F5000AA2797FDA095BA2F840F951FA61FB71F0C
:102F600080931A0490931B04A0931C04B0931D0437
:102F700040911E0450911F0460912004709121041F
:102F80002091D2033091D303C901880F991F820F7A
:102F9000931F880F991F880F991FAA2797FDA09547
:102FA000BA2F840F951FA61FB71F80931E049093FE
:102FB0001F04A0932004B093210460912204709117
:102FC00023048091240490912504E090FD06F09064
:102FD000FE06A0900404B0900504C0900604D090B2
:102FE00007040E94B03B3B014C010027F7FC009511
:102FF000102FC801B7010E94B03BA60195010E94A5
:10300000AC3A9B01AC01C401B3010E94AD3A0E94ED
:103010007D3B609322047093230480932404909357
:10302000250420913A0430913B0440913C04509196
:103030003D048091B0079091B107AA2797FDA09514
:10304000BA2F820F931FA41FB51F80933A04909349
:103050003B04A0933C04B0933D0420913E04309186
:103060003F0440914004509141048091B0079091F9
:10307000B107AA2797FDA095BA2F820F931FA41F0F
:10308000B51F80933E0490933F04A0934004B093F7
:103090004104209168042A83222309F069C08091A9
:1030A0006904882309F064C08091490786FF60C0E5
:1030B00060912A0470912B0480912C0490912D042E
:1030C000E090B007F090B107A0907604BB24CC2428
:1030D000DD240027F7FC0095102F20E030E140E0D0
:1030E00050E00E943B3DC801B7010E94C73CA601C9
:1030F00095010E94C73C20E038E040E050E00E948B
:103100003B3D2093C5043093C6044093C7045093BD
:10311000C80460913204709133048091340490911A
:103120003504E090B007F090B10720E030E140E0D6
:1031300050E00E943B3DCA01B901A60195010E94E1
:10314000C73C0027F7FC0095102FA80197010E94AB
:10315000C73C20E038E040E050E00E943B3D209337
:10316000C1043093C2044093C3045093C40410C0FC
:103170001092C1041092C2041092C3041092C404AD
:103180001092C5041092C6041092C7041092C8048D
:103190008091890790918A072090C5043090C604D9
:1031A0004090C7045090C804820D931D90938A07E5
:1031B000809389070091890710918A07A090C10424
:1031C000B090C204C090C304D090C404809177042E
:1031D000682E772488249924C401B301A60195019F
:1031E0000E94C73C20E032E040E050E00E943B3DBE
:1031F000020F131F10938A0700938907209136044A
:1032000030913704409138045091390480918907F6
:1032100090918A07AA2797FDA095BA2F820F931F36
:10322000A41FB51F8093360490933704A0933804ED
:10323000B0933904409132045091330460913404C6
:10324000709135048091890790918A0720916404D8
:1032500030916504821B930BAA2797FDA095BA2F86
:10326000840F951FA61FB71F8093320490933304D9
:10327000A0933404B09335048091320490913304C8
:10328000A0913404B0913504E0908C03F0908D034C
:1032900000918E0310918F03E816F9060A071B07A9
:1032A00004F580E197E2A0E0B0E08E199F09A00B41
:1032B000B10B8093320490933304A0933404B09301
:1032C00035048091320490913304A0913404B0917C
:1032D00035048093360490933704A0933804B09358
:1032E00039042091320430913304409134045091D8
:1032F000350488279927DC018E199F09A00BB10B93
:10330000281739074A075B0704F580EF98EDAFEF00
:10331000BFEFE80EF91E0A1F1B1FE0923204F09265
:103320003304009334041093350480913204909157
:103330003304A0913404B091350480933604909303
:103340003704A0933804B09339048091CE03909150
:10335000CF030F9734F488E19CEF90938A07809312
:1033600089078091CE039091CF03079734F480E3CF
:1033700098EF90938A078093890790910001998331
:103380009A30A9F48091CE039091CF03835F93404C
:1033900034F088EE93E090938A07809389078091B8
:1033A000CE039091CF038A5F9340DCF014C08091EC
:1033B000CE039091CF03855E974034F088EE93E082
:1033C00090938A07809389078091CE039091CF03D1
:1033D000835F974034F080ED97E090938A07809365
:1033E000890780919107909192078A199B09909380
:1033F0009207809391070091910710919207C40161
:10340000B301A20191010E94C73C20E032E040E0FC
:1034100050E00E943B3D50954095309521953F4F9F
:103420004F4F5F4F020F131F1093920700939107A6
:1034300020912E0430912F0440913004509131049A
:103440008091910790919207AA2797FDA095BA2F96
:10345000820F931FA41FB51F80932E0490932F04F7
:10346000A0933004B093310440912A0450912B046E
:1034700060912C0470912D04809191079091920796
:103480002091660430916704821B930BAA2797FD55
:10349000A095BA2F840F951FA61FB71F80932A04EB
:1034A00090932B04A0932C04B0932D0480912A04B4
:1034B00090912B04A0912C04B0912D04E0908803EE
:1034C000F090890300918A0310918B03E816F906A6
:1034D0000A071B0704F580E197E2A0E0B0E08E192F
:1034E0009F09A00BB10B80932A0490932B04A09307
:1034F0002C04B0932D0480912A0490912B04A09168
:103500002C04B0912D0480932E0490932F04A0934B
:103510003004B093310420912A0430912B0440915F
:103520002C0450912D0488279927DC018E199F09BE
:10353000A00BB10B281739074A075B0704F580EF8A
:1035400098EDAFEFBFEFE80EF91E0A1F1B1FE092C8
:103550002A04F0922B0400932C0410932D048091E4
:103560002A0490912B04A0912C04B0912D048093F7
:103570002E0490932F04A0933004B09331048091D3
:10358000CC039091CD030F9734F488E19CEF909396
:103590009207809391078091CC039091CD03079778
:1035A00034F480E398EF9093920780939107998188
:1035B0009A30A9F48091CC039091CD03835F93401E
:1035C00034F088EE93E09093920780939107809176
:1035D000CC039091CD038A5F9340DCF014C08091BE
:1035E000CC039091CD03855E974034F088EE93E054
:1035F00090939207809391078091CC039091CD0393
:10360000835F974034F080ED97E09093920780932A
:1036100091078FEE80937A0080913A0490913B0459
:10362000A0913C04B0913D0480932604909327041C
:10363000A0932804B093290480912A0490912B042C
:10364000A0912C04B0912D0480930A0490930B0454
:10365000A0930C04B0930D04809132049091330434
:10366000A0913404B0913504809312049093130414
:10367000A0931404B093150480912E0490912F040C
:10368000A0913004B091310480930E0490930F0404
:10369000A0931004B09311048091360490913704E4
:1036A000A0913804B09139048093160490931704C4
:1036B000A0931804B09319048091490787FF63C051
:1036C0002A81222309F05FC080916904882309F0D0
:1036D0005AC08091910790919207893C91055CF0C6
:1036E00020919107309192078091910790919207D4
:1036F000885C904011C08091910790919207885307
:103700009F4FA4F4209191073091920780919107E7
:103710009091920788539F4F880F991F880F991F88
:10372000820F931F9093920780939107809189074E
:1037300090918A07893C91055CF02091890730912E
:103740008A078091890790918A07885C904011C010
:103750008091890790918A0788539F4FA4F4209104
:10376000890730918A078091890790918A07885349
:103770009F4F880F991F880F991F820F931F909357
:103780008A078093890780914507E82FF0E0EE0FC4
:10379000FF1FEB5EF84F8081918120914E043091A4
:1037A0004F0483599F4F821793071CF02F5F3F4FA1
:1037B0000CC08081918182599F4F821793074CF4EE
:1037C0002115310531F02150304030934F042093C2
:1037D0004E0480914607E82FF0E0EE0FFF1FEB5EEE
:1037E000F84F808191812091500430915104835988
:1037F0009F4F821793071CF02F5F3F4F0CC08081B3
:10380000918182599F4F821793074CF421153105FE
:1038100031F0215030403093510420935004809176
:103820004707E82FF0E0EE0FFF1FEB5EF84F8081B7
:103830009181209152043091530483599F4F8217F4
:1038400093071CF02F5F3F4F0CC0808191818259FC
:103850009F4F821793074CF42115310531F0215009
:103860003040309353042093520480914807E82F4E
:10387000F0E0EE0FFF1FEB5EF84F80819181209109
:1038800054043091550483599F4F821793071CF0BD
:103890002F5F3F4F0CC08081918182599F4F8217CB
:1038A00093074CF42115310531F02150304030930D
:1038B00055042093540480914E0490914F0497FF37
:1038C00005C010924F0410924E040AC08F3F91051C
:1038D00039F034F08FEF90E090934F0480934E04D2
:1038E000809150049091510497FF05C010925104AB
:1038F000109250040AC08F3F910539F034F08FEFD9
:1039000090E09093510480935004809152049091E0
:10391000530497FF05C010925304109252040AC03A
:103920008F3F910539F034F08FEF90E0909353047E
:1039300080935204809154049091550497FF05C0E0
:1039400010925504109254040AC08F3F910539F02B
:1039500034F08FEF90E090935504809354040F90CF
:103960000F90CF91DF911F910F91FF90EF90DF901B
:10397000CF90BF90AF909F908F907F906F905F900F
:103980004F903F902F90089510927A008091CC0331
:103990009091CD0390939207809391078091CE03ED
:1039A0009091CF0390938A07809389078091D003E9
:1039B0009091D1039093B1078093B0076091D403A5
:1039C0007091D503882777FD8095982F2CE030E003
:1039D00040E050E00E94C73C7093AE076093AD0793
:1039E0006091D2037091D303882777FD8095982F3B
:1039F0000E94C73C7093B8076093B7078091D603C5
:103A00009091D70390939907809398078FEE8093B6
:103A10007A0080914507E82FF0E0EE0FFF1FEB5E84
:103A2000F84F8081918120914E0430914F04835949
:103A30009F4F821793071CF02F5F3F4F0CC0808170
:103A4000918182599F4F821793074CF421153105BC
:103A500031F02150304030934F0420934E04809138
:103A60004607E82FF0E0EE0FFF1FEB5EF84F808176
:103A70009181209150043091510483599F4F8217B6
:103A800093071CF02F5F3F4F0CC0808191818259BA
:103A90009F4F821793074CF42115310531F02150C7
:103AA0003040309351042093500480914707E82F11
:103AB000F0E0EE0FFF1FEB5EF84F808191812091C7
:103AC00052043091530483599F4F821793071CF07F
:103AD0002F5F3F4F0CC08081918182599F4F821789
:103AE00093074CF42115310531F0215030403093CB
:103AF00053042093520480914807E82FF0E0EE0F22
:103B0000FF1FEB5EF84F808191812091540430912A
:103B1000550483599F4F821793071CF02F5F3F4F27
:103B20000CC08081918182599F4F821793074CF47A
:103B30002115310531F02150304030935504209348
:103B4000540480914E0490914F0497FF05C0109249
:103B50004F0410924E040AC08F3F910539F034F0A3
:103B60008FEF90E090934F0480934E048091500427
:103B70009091510497FF05C0109251041092500487
:103B80000AC08F3F910539F034F08FEF90E09093A9
:103B9000510480935004809152049091530497FFF4
:103BA00005C010925304109252040AC08F3F910531
:103BB00039F034F08FEF90E09093530480935204E7
:103BC000809154049091550497FF05C010925504BC
:103BD000109254040AC08F3F910539F034F08FEFF2
:103BE00090E0909355048093540460916C0770E0CA
:103BF00080E090E024EC39E040E050E00E94C73CD7
:103C0000609388037093890380938A0390938B0356
:103C100060938C0370938D0380938E0390938F0336
:103C2000089580914C078B3F98F08B3F19F4809159
:103C30004E040EC08C3F19F48091500409C08D3F92
:103C400019F48091520404C08E3F21F480915404F1
:103C50008093950380919503882319F4109295031E
:103C600004C08F3F11F48093950380914B078B3FE5
:103C700098F08B3F19F480914E040EC08C3F19F4DC
:103C80008091500409C08D3F19F48091520404C002
:103C90008E3F21F480915404809394038091940387
:103CA000882319F41092940305C0843618F084E632
:103CB0008093940380914D078B3F98F08B3F19F4CC
:103CC00080914E040EC08C3F19F48091500409C0BD
:103CD0008D3F19F48091520404C08E3F21F48091ED
:103CE00054048093960380919603882319F41092CC
:103CF000960305C0843618F084E68093960380917D
:103D00004F078B3F98F08B3F19F480914E040EC003
:103D10008C3F19F48091500409C08D3F19F48091B3
:103D2000520404C08E3F21F4809154048093970381
:103D300080919703882319F41092970304C08F3F52
:103D400011F480939703809156078B3F98F08B3F37
:103D500019F480914E040EC08C3F19F480915004E8
:103D600009C08D3F19F48091520404C08E3F21F4A4
:103D7000809154048093980380919803882319F4C8
:103D80001092980304C08F3F11F4809398038091A0
:103D900057078B3F98F08B3F19F480914E040EC06B
:103DA0008C3F19F48091500409C08D3F19F4809123
:103DB000520404C08E3F21F48091540480939903EF
:103DC000809199038B3010F48AE002C08F3F11F488
:103DD00080939903809158078B3F98F08B3F19F49B
:103DE00080914E040EC08C3F19F48091500409C09C
:103DF0008D3F19F48091520404C08E3F21F48091CC
:103E0000540480939A0380919A03882319F41092A2
:103E10009A0304C08F3F11F480939A0380915D0749
:103E20008B3F98F08B3F19F480914E040EC08C3F6D
:103E300019F48091500409C08D3F19F48091520407
:103E400004C08E3F21F48091540480939C038091A0
:103E50009C03882319F410929C0304C08F3F11F433
:103E600080939C0380915E078B3F98F08B3F19F401
:103E700080914E040EC08C3F19F48091500409C00B
:103E80008D3F19F48091520404C08E3F21F480913B
:103E9000540480936E0480916E04882319F4109268
:103EA0006E0404C08F3F11F480936E0480915F070D
:103EB0008B3F98F08B3F19F480914E040EC08C3FDD
:103EC00019F48091500409C08D3F19F48091520477
:103ED00004C08E3F21F48091540480936F0480913C
:103EE0006F04882319F410926F0404C08F3F11F4FB
:103EF00080936F04809160078B3F98F08B3F19F49B
:103F000080914E040EC08C3F19F48091500409C07A
:103F10008D3F19F48091520404C08E3F21F48091AA
:103F200054048093700480917004882319F41092D3
:103F3000700404C08F3F11F4809370048091610776
:103F40008B3F98F08B3F19F480914E040EC08C3F4C
:103F500019F48091500409C08D3F19F480915204E6
:103F600004C08E3F21F480915404809371048091A9
:103F70007104882319F41092710404C08F3F11F466
:103F800080937104809171078B3F98F08B3F19F4F7
:103F900080914E040EC08C3F19F48091500409C0EA
:103FA0008D3F19F48091520404C08E3F21F480911A
:103FB00054048093720480917204882319F410923F
:103FC000720404C08F3F11F48093720480917207D1
:103FD0008B3F98F08B3F19F480914E040EC08C3FBC
:103FE00019F48091500409C08D3F19F48091520456
:103FF00004C08E3F21F48091540480937304809117
:104000007304882319F41092730404C08F3F11F4D1
:1040100080937304809173078B3F98F08B3F19F462
:1040200080914E040EC08C3F19F48091500409C059
:104030008D3F19F48091520404C08E3F21F4809189
:1040400054048093740480917404882319F41092AA
:10405000740404C08F3F11F480937404809174073A
:104060008B3F98F08B3F19F480914E040EC08C3F2B
:1040700019F48091500409C08D3F19F480915204C5
:1040800004C08E3F21F48091540480937504809184
:104090007504882319F41092750404C08F3F11F43D
:1040A00080937504809162078B3F98F08B3F19F4E1
:1040B00080914E040EC08C3F19F48091500409C0C9
:1040C0008D3F19F48091520404C08E3F21F48091F9
:1040D000540480939D0380919D03882319F41092CA
:1040E0009D0304C08F3F11F480939D038091670767
:1040F0008B3F98F08B3F19F480914E040EC08C3F9B
:1041000019F48091500409C08D3F19F48091520434
:1041100004C08E3F21F48091540480939E038091CB
:104120009E03882319F410929E0304C08F3F11F45C
:1041300080939E0380916A078B3F98F08B3F19F420
:1041400080914E040EC08C3F19F48091500409C038
:104150008D3F19F48091520404C08E3F21F4809168
:1041600054048093760480917604882319F4109285
:10417000760404C08F3F11F48093760480916B071E
:104180008B3F98F08B3F19F480914E040EC08C3F0A
:1041900019F48091500409C08D3F19F480915204A4
:1041A00004C08E3F21F48091540480937704809161
:1041B0007704882319F41092770404C08F3F11F418
:1041C00080937704809170078B3F98F08B3F19F4B0
:1041D00080914E040EC08C3F19F48091500409C0A8
:1041E0008D3F19F48091520404C08E3F21F48091D8
:1041F000540480939F0380919F03882319F41092A5
:104200009F0304C08F3F11F480939F0360919C0330
:1042100070E080E090E00E94AE3B27E137EB41ED9B
:1042200058E30E94643C60939003709391038093E1
:10423000920390939303809154078093AF078091EA
:10424000530780939307089580915F04882301F5B5
:104250001092900710928B071092A8071092AA074D
:104260008091B003882311F080938B078091B10374
:10427000882311F0809390078091B203882311F076
:104280008093AA078091B303882311F08093A80735
:1042900080918B07E1EDF6E08093D1061092D20673
:1042A000809190078093D30613828091AA07809310
:1042B000D50615828091A8078093D70617821092A1
:1042C000EF031092F0030E94281508951092010444
:1042D00010920004109203041092020480E090E017
:1042E000A0E0B0E08093040490930504A09306043A
:1042F000B09307041092F7031092F6031092F9039B
:104300001092F8031092FB031092FA0310927604B5
:10431000109277040E94C41C84E690E00E94C20CB4
:104320000E94C41C8091490780FF10C080910F0338
:1043300090911003875B934038F480910F03909124
:1043400010038E5E924010F40E941C108091CC03EA
:104350009091CD039093F7038093F6038091CE0361
:104360009091CF039093F9038093F8038091D00349
:104370009091D1039093FB038093FA038091F8030B
:104380009091F9039093FD038093FC038091F603D1
:104390009091F7039093FF038093FE03F999FECF6A
:1043A00024E030E032BD21BDF89A80B5853038F187
:1043B0008091B7079091B80797FF03C090958195BA
:1043C0009F4F6CE070E00E94063D70930304609381
:1043D00002048091AD079091AE0797FF03C09095BE
:1043E00081959F4F6CE070E00E94063D7093010440
:1043F000609300046091FD067091FE0642C0F99939
:10440000FECF32BD21BDF89A30B5F999FECF85E0D7
:1044100090E092BD81BDF89A20B5932F80E0820F85
:10442000911D9093010480930004F999FECF86E0DA
:1044300090E092BD81BDF89A30B5F999FECF87E042
:1044400090E092BD81BDF89A20B5932F80E0820F55
:10445000911D9093030480930204F999FECF88E0A4
:1044600090E092BD81BDF89A30B5F999FECF89E010
:1044700090E092BD81BDF89A20B5732F60E0620F85
:10448000711D882777FD8095982F0E94B03B60931F
:10449000040470930504809306049093070410921B
:1044A0002A0410922B0410922C0410922D041092C6
:1044B0002E0410922F0410923004109231041092A6
:1044C0003204109233041092340410923504109286
:1044D0003604109237041092380410923904109266
:1044E0003A0410923B0410923C0410923D04109246
:1044F00092071092910710928A07109289071092E2
:10450000B1071092B00780910B0390910C03A0911A
:104510000D03B0910E03909300078093FF06109255
:10452000DF031092DE0310924204109243041092B3
:10453000440410924504809146049091470490935E
:104540004904809348040E943D3A82E390E09093AE
:10455000C6038093C50360916C0770E080E090E033
:1045600024EC39E040E050E00E94C73C60938803AF
:104570007093890380938A0390938B0360916D07F6
:1045800070E080E090E00E94C73C60938C037093E1
:104590008D0380938E0390938F031092A10310924A
:1045A000A00308951F93CF93DF93182FC4E6D0E0A4
:1045B0000DC0115080915F04882351F4D093C6033D
:1045C000C093C5038AEF90E00E94AC0C112389F7D9
:1045D000DF91CF911F9108952F923F924F925F925A
:1045E0006F927F928F929F92AF92BF92CF92DF9203
:1045F000EF92FF920F931F93DF93CF93CDB7DEB768
:1046000028970FB6F894DEBF0FBECDBF0E94E2160A
:10461000299A80915D0490915E049C013A832983DC
:1046200037FF02C01A82198280915604843608F03E
:1046300061C0809103018823B9F480E090E00E947A
:104640006D0C80910403909105038F5F9F4F61F47F
:1046500088E99AE39093C6038093C50380E09CE0C9
:1046600090930503809304038091A3049091A40484
:10467000009731F001979093A4048093A30404C0A1
:1046800010925F0410924C04809100018A3011F462
:10469000289A01C0289880919E0490919F04815D82
:1046A000974028F180915A07482F50E05A83498358
:1046B00081E080934C04E0914107F0E0EE0FFF1F92
:1046C000EB5EF84F11821082E0914207F0E0EE0FAE
:1046D000FF1FEB5EF84F11821082E0914407F0E07B
:1046E000EE0FFF1FEB5EF84F11821082AEC21092E8
:1046F0005F04ABC2809156048D3808F4A6C21092B4
:104700004C0480915B0722E3829FC00111249093A7
:10471000A4048093A30469817A81693271056CF0E5
:1047200080919E0490919F047FEF8F3F970729F01F
:10473000019690939F0480939E0480919E04909193
:104740009F04883C910520F089819A81889704F51F
:104750001092BD041092BE041092BF041092C004C7
:104760001092B9041092BA041092BB041092BC04C7
:1047700010923A0410923B0410923C0410923D04B3
:1047800010923E0410923F04109240041092410493
:10479000E0914307F0E0EE0FFF1FEB5EF84F8081E2
:1047A0009181813591050CF49CC180915F0488232F
:1047B00009F097C180914407E82FF0E0EE0FFF1F4A
:1047C000EB5EF84F808191818C3491050CF4C8C068
:1047D0008091A2048F5F8093A204893C08F481C178
:1047E000299810925F041092A20410929F041092D4
:1047F0009E0480914107482F50E0FA01EE0FFF1F01
:10480000EB5EF84F80819181873491059CF4E091B3
:104810004207F0E0EE0FFF1FEB5EF84F0190F081D2
:10482000E02DF7FF03C0F095E195FF4FE734F10568
:104830000CF478C080914207A82FB0E0FD01EE0F84
:10484000FF1FEB5EF84F808191818734910544F022
:10485000FA01EE0FFF1FEB5EF84F0190F081E02DA3
:10486000FD01EE0FFF1FEB5EF84F808191818734D1
:10487000910564F0FA01EE0FFF1FEB5EF84F8081A7
:1048800091818734910514F022E001C021E0FD01FF
:10489000EE0FFF1FEB5EF84F80819181863491050A
:1048A0005CF4FA01EE0FFF1FEB5EF84F80819181FF
:1048B000873491050CF023E0FD01EE0FFF1FEB5E46
:1048C000F84F808191818A5B9F4F5CF4FA01EE0F73
:1048D000FF1FEB5EF84F80819181873491050CF0CA
:1048E00024E0AA0FBB1FAB5EB84F8D919C918A5BF1
:1048F0009F4F5CF4440F551F4B5E584FDA018D916A
:104900009C91863491050CF425E0F999FECF1FBAED
:1049100082E090E092BD81BD20BD0FB6F894FA9A76
:10492000F99A0FBE8091490780FF10C080910F0354
:1049300090911003875B934038F480910F0390911E
:1049400010038E5E924010F40E941C100E946D02B3
:1049500047E461E477E00E94A2020E946621BAC0A7
:1049600080819181855B9F4F0CF0B9C08091A2043A
:104970008F5F8093A204893C08F4B3C02998F99909
:10498000FECF1FBA04E010E012BD01BD8FEF80BD65
:104990000FB6F894FA9AF99A0FBE10925F0410922B
:1049A000A20410929F0410929E040E94662180919E
:1049B000000490910104F999FECF1FBA12BD01BD08
:1049C00060E071E00E94063D60BD0FB6F894FA9A6F
:1049D000F99A0FBE2091000430910104F999FECF9D
:1049E0001FBA85E090E092BD81BDC90160E071E031
:1049F0000E94063D80BD0FB6F894FA9AF99A0FBE50
:104A00002091020430910304F999FECF1FBA86E089
:104A100090E092BD81BDC90160E071E00E94063D59
:104A200060BD0FB6F894FA9AF99A0FBE209102046D
:104A300030910304F999FECF1FBA87E090E092BD50
:104A400081BDC90160E071E00E94063D80BD0FB6E6
:104A5000F894FA9AF99A0FBE209104043091050453
:104A60004091060450910704F999FECF1FBA88E0DF
:104A700090E092BD81BDCA01B9010E947D3BDC017D
:104A8000CB0160E071E00E94063D60BD0FB6F89476
:104A9000FA9AF99A0FBE20910404309105044091CE
:104AA000060450910704F999FECF1FBA89E090E0FF
:104AB00092BD81BDCA01B9010E947D3BDC01CB01E1
:104AC00060E071E00E94063D80BD0FB6F894FA9A4E
:104AD000F99A0FBE0E946D020E94D22202C010926B
:104AE000A204E0914307F0E0EE0FFF1FEB5EF84FEA
:104AF000808191818B5A9F4F0CF0A7C0E0914407B1
:104B0000F0E0EE0FFF1FEB5EF84F80819181855B37
:104B10009F4F0CF07AC0E0914807F0E0EE0FFF1FC6
:104B2000EB5EF84F80819181893791050CF46DC05F
:104B30008091A1048F5F8093A104893C08F467C031
:104B400088EC8093A10481E090E090939F0480938F
:104B50009E0481E080935F041092B5041092B60425
:104B60001092B7041092B80410923A0410923B04C9
:104B700010923C0410923D0410923E0410923F04A7
:104B8000109240041092410410922A0410922B04B7
:104B900010922C0410922D041092320410923304BF
:104BA000109234041092350480910A0490910B0401
:104BB000A0910C04B0910D0480932E0490932F04C7
:104BC000A0933004B09331048091120490911304A7
:104BD000A0911404B0911504809336049093370487
:104BE000A0933804B09339041092BD041092BE040F
:104BF0001092BF041092C0041092B9041092BA042B
:104C00001092BB041092BC0402C01092A104E09167
:104C10004807F0E0EE0FFF1FEB5EF84F80819181B7
:104C200044978CF48091A0048F5F8093A004853614
:104C300060F010925F0484E68093A00410929F04B9
:104C400010929E0402C01092A00480916C038150C7
:104C500080936C038F5F29F080914C04882309F4C2
:104C600090C30E94111E80914107882E9924F4015F
:104C7000EE0FFF1FB5E1CB2EB7E0DB2ECE0EDF1E11
:104C8000D6018D919C91E0905007FF249C012E9DB0
:104C9000C0012F9D900D3E9D900D11244091570411
:104CA000509158049A01220F331F240F351F820F91
:104CB000931F64E070E00E94063DCB01709358049E
:104CC00060935704E55DF84F2081318100915107D1
:104CD00010E0A901409F9001419F300D509F300D81
:104CE0001124820F931F90935804809357042091AE
:104CF0004207A22EBB24AA0CBB1CF501EB5EF84FA9
:104D000080819181BC016E9DC0016F9D900D7E9D43
:104D1000900D11244091590450915A049A01220F88
:104D2000331F240F351F820F931F64E070E00E9431
:104D3000063DCB0170935A0460935904ABE2B7E08F
:104D4000AA0EBB1EF50120813181A901409F90016F
:104D5000419F300D509F300D1124820F931F90936F
:104D60005A0480935904E0914407F0E0EE0FFF1FCE
:104D7000EB5EF84F80819181909581959F4F909344
:104D80005C0480935B04E0914307F0E0EE0FFF1FAB
:104D9000EB5EF84F8081918188589F4F90935E041D
:104DA00080935D04D6018D919C9120917E04309179
:104DB0007F0497FF03C0909581959F4F281739076F
:104DC000C4F4880C991CE5E1F7E08E0E9F1ED40117
:104DD000ED91FC91F0937F04E0937E04F7FF0FC008
:104DE000882799278E1B9F0B90937F0480937E04C6
:104DF00006C02150304030937F0420937E04809180
:104E00004207A82FB0E0FD01EE0FFF1FEB5EF84F49
:104E100080819181209180043091810497FF03C0AB
:104E2000909581959F4F28173907ACF4AA0FBB1FA7
:104E3000AB5EB84FED91FC91F0938104E093800458
:104E4000F7FF0FC0882799278E1B9F0B9093810433
:104E50008093800406C02150304030938104209319
:104E6000800480914C04882341F010927F041092BA
:104E70007E0410928104109280046091990370E086
:104E800080E090E00E94AE3B20E030E040E251E460
:104E90000E94AD3A20E030E040E85BE30E94643CD1
:104EA0006093B2077093B3078093B4079093B507EC
:104EB00060919A0370E080E090E00E94AE3B20E0B9
:104EC00030EE4BE257E40E94153B6093A4077093C9
:104ED000A5078093A6079093A7078091B503882321
:104EE00031F08AE090E09093C6038093C5038091EF
:104EF000B50382FF09C080916E04482F50E0440F33
:104F0000551F440F551F10C083FD03C040E050E003
:104F10000BC080916E0490E0880F991F880F991F35
:104F200044275527481B590B209178043091790468
:104F3000C901F3E0880F991FFA95E1F7821B930BE3
:104F4000840F951F68E070E00E94063D709379041D
:104F5000609378048091B50384FF09C080916E044A
:104F6000482F50E0440F551F440F551F10C085FDBA
:104F700003C040E050E00BC080916E0490E0880FC9
:104F8000991F880F991F44275527481B590B2091BB
:104F90007A0430917B04C90163E0880F991F6A95F8
:104FA000E1F7821B930B840F951F68E070E00E946D
:104FB000063D70937B0460937A048091B40383FF71
:104FC00003C082E390E004C082FF07C08EEC9FEF35
:104FD00090937D0480937C0404C010927D04109211
:104FE0007C048091B40381FF09C08091A00390915B
:104FF000A10301969093A1038093A0038091B40331
:1050000084FF09C08091A0039091A1030197909320
:10501000A1038093A003809178049091790468E0C3
:1050200070E00E94063DE0915704F0915804E60FAD
:10503000F71FF0935804E093570480917A049091FD
:105040007B0468E070E00E94063D40915904509155
:105050005A04460F571F50935A04409359046091C5
:105060005B0470915C0480917C0490917D04680FD6
:10507000791F70935C0460935B048091200680FF2D
:105080005CC080916E04813808F457C020915007AD
:1050900030E080911906992787FD9095DC012A9FC1
:1050A000C0012B9F900D3A9F900D1124E80FF91F1E
:1050B000F0935804E093570480911A06992787FDCE
:1050C0009095FC012E9FC0012F9F900D3E9F900D4B
:1050D0001124480F591F50935A044093590480914A
:1050E0001B06992787FD9095680F791F70935C04C4
:1050F00060935B0420914E0730E080911D06992754
:1051000087FD9095AC01249FC001259F900D349F91
:10511000900D11249093A1038093A00380911C060D
:10512000282F30E080915D0490915E0428173907A4
:1051300024F430935E0420935D048091490782FF3C
:105140000CC080E090E0A0E0B0E08093A4079093D2
:10515000A507A093A607B093A70720E030E040E0A2
:1051600050E06091B2077091B3078091B4079091BD
:10517000B5070E94113B882364F480E090E0A0E032
:10518000B0E08093B2079093B307A093B407B093B5
:10519000B50720E030E040E050E06091A407709156
:1051A000A5078091A6079091A7070E94113B88232D
:1051B00064F480E090E0A0E0B0E08093A4079093D6
:1051C000A507A093A607B093A70780914207A82F31
:1051D000B0E0FD01EE0FFF1FEB5EF84F2081318143
:1051E00080916807482F50E04217530744F480919C
:1051F000750782FF04C081E080936A040FC0AA0F84
:10520000BB1FAB5EB84F2D913C9180916907481B45
:1052100051092417350714F410926A04809142074B
:10522000A82FB0E0FD01EE0FFF1FEB5EF84F2081CD
:10523000318180916807482F50E088279927841B87
:10524000950B2817390744F48091750783FF04C034
:1052500081E080936B0414C080916B04882381F0FB
:10526000AA0FBB1FAB5EB84F2D913C91809169078F
:1052700090E0841B950B8217930714F410926B0433
:1052800080914107A82FB0E0FD01EE0FFF1FEB5EFC
:10529000F84F2081318180916807482F50E04217F4
:1052A000530744F48091750780FF04C081E0809328
:1052B0006D0413C080916D04882379F0AA0FBB1F81
:1052C000AB5EB84F2D913C9180916907481B510905
:1052D0002417350714F410926D0480914107A82F0C
:1052E000B0E0FD01EE0FFF1FEB5EF84F2081318132
:1052F00080916807482F50E088279927841B950BD9
:105300002817390744F48091750781FF04C081E0B4
:1053100080936C0414C080916C04882381F0AA0FE0
:10532000BB1FAB5EB84F2D913C918091690790E017
:10533000841B950B8217930714F410926C048091D0
:105340006A04882321F480916B04882321F081E092
:105350008093690402C01092690480916D048823CF
:1053600021F480916C04882351F081E080936804DB
:105370001092690410926A0410926B0402C0109299
:10538000680480916904882331F084E690E090936A
:10539000C6038093C50380916904882321F480911A
:1053A0006804882351F08091670790E069817A81D1
:1053B0008617970714F49A83898380914C04882375
:1053C00041F110925C0410925B0410925804109208
:1053D000570410925A04109259048DEC9CECACECDA
:1053E000BDE38093B2079093B307A093B407B09343
:1053F000B5078AE097EDA3EABBE38093A4079093F7
:10540000A507A093A607B093A7071092690410926E
:10541000680420919C0730919D0740919E07509110
:105420009F0780910A0490910B04A0910C04B09105
:105430000D04820F931FA41FB51F80939C079093A8
:105440009D07A0939E07B0939F072091A0073091DE
:10545000A1074091A2075091A30780911204909157
:105460001304A0911404B0911504820F931FA41F7C
:10547000B51F8093A0079093A107A093A207B093B4
:10548000A30720919407309195074091960750917A
:10549000970780910E0490910F04A0911004B09191
:1054A0001104820F931FA41FB51F8093940790933C
:1054B0009507A0939607B093970720918C0730919A
:1054C0008D0740918E0750918F078091160490911F
:1054D0001704A0911804B0911904820F931FA41F00
:1054E000B51F80938C0790938D07A0938E07B09380
:1054F0008F0780916804882329F4809169048823A8
:1055000009F45CC010921A0410921B0410921C043F
:1055100010921D0410921E0410921F041092200479
:105520001092210410929C0710929D0710929E07E2
:1055300010929F071092A0071092A1071092A20745
:105540001092A30710929407109295071092960755
:105550001092970710928C0710928D0710928E0769
:1055600010928F0780912A0490912B04A0912C0413
:10557000B0912D0480932E0490932F04A0933004B7
:10558000B09331048091320490913304A09134049B
:10559000B09135048093360490933704A093380477
:1055A000B09339041092E1031092E0031092670463
:1055B000109266041092650410926404809168044D
:1055C000882309F015C180916904882309F010C16E
:1055D00060910A0470910B0480910C0490910D0469
:1055E000A0905507BB24CC24DD24E090AD07F090BB
:1055F000AE07A60195010E943B3D39014A010027F3
:10560000F7FC0095102F6E187F08800A910A6091B0
:105610001204709113048091140490911504E09089
:10562000B707F090B807A60195010E943B3D5901CC
:105630006A010027F7FC0095102FAE18BF08C00ABA
:10564000D10AC401B30120E130E040E050E00E9403
:105650003B3D522E432E342E252E822F932FA42FE6
:10566000B52F3C014D01C601B50120E130E040E01D
:1056700050E00E943B3DC22EA32ED42EB52E822F89
:10568000932FA42FB52F7C018D0180917E049091E2
:105690007F04409734F48091800490918104409776
:1056A000E4F0652D742D832D922D23E030E040E051
:1056B00050E00E943B3DC901DA013C014D016C2DD7
:1056C0007A2D8D2D9B2D23E030E040E050E00E94AC
:1056D0003B3DC901DA017C018D01E0914407F0E016
:1056E000EE0FFF1FEB5EF84F0190F081E02DF7FF0A
:1056F00003C0F095E195FF4F7A97C4F0C401B30160
:1057000023E030E040E050E00E943B3DC901DA0177
:105710003C014D01C801B70123E030E040E050E01A
:105720000E943B3DC901DA017C018D0171E26716DF
:1057300071048104910434F020E2622E712C812CDA
:10574000912C11C080EE68168FEF78068FEF8806D7
:105750008FEF980644F490EE692E9FEF792E9FEF1D
:10576000892E9FEF992E91E2E916F10401051105AA
:1057700034F080E2E82EF12C012D112D11C0A0EEA5
:10578000EA16AFEFFA06AFEF0A07AFEF1A0744F4D5
:1057900000EEE02E0FEFF02E0FEF002F0FEF102F87
:1057A00080912A0490912B04A0912C04B0912D0497
:1057B00086199709A809B90980932A0490932B04A4
:1057C000A0932C04B0932D04809132049091330463
:1057D000A0913404B09135048E199F09A00BB10B30
:1057E0008093320490933304A0933404B09335042F
:1057F0008091E0039091E1038F3F910509F008F457
:1058000085C580916804882309F004C580916904E6
:10581000882309F0FFC460919C0770919D078091D7
:105820009E0790919F0720E031E040E050E00E9409
:105830003B3DC901DA0180939C0790939D07A0939B
:105840009E07B0939F076091A0077091A107809178
:10585000A2079091A30720E031E040E050E00E94D1
:105860003B3DC901DA018093A0079093A107A09363
:10587000A207B093A30720911A0430911B04409112
:105880001C0450911D04E0905507FF2400E010E037
:10589000C801B7010E94C73C20E031E040E050E081
:1058A0000E943B3DC901DA0180931A0490931B04C6
:1058B000A0931C04B0931D0420911E0430911F047A
:1058C0004091200450912104C801B7010E94C73CB7
:1058D00020E031E040E050E00E943B3DC901DA01A8
:1058E00080931E0490931F04A0932004B09321047E
:1058F00060912204709123048091240490912504E6
:1059000020E031E040E050E00E943B3DC901DA0177
:105910008093220490932304A0932404B09325043D
:1059200060919C0770919D0780919E0790919F07C1
:1059300020911A0430911B0440911C0450911D04C5
:10594000621B730B840B950B6093A9047093AA04DC
:105950008093AB049093AC04E0906E07FF2400E0CA
:1059600010E0A80197010E943B3D59016A01209374
:10597000960430939704409398045093990460914F
:10598000A0077091A1078091A2079091A307209191
:105990001E0430911F044091200450912104621B89
:1059A000730B840B950B6093A5047093A6048093EE
:1059B000A7049093A804A80197010E943B3D790198
:1059C0008A0120939204309393044093940450935B
:1059D0009504C601B50120E031E040E050E00E94AE
:1059E0003B3D3093670420936604C801B70120E073
:1059F00031E040E050E00E943B3D3093650420934D
:105A0000640480917E0490917F044097BCF480915F
:105A100080049091810440978CF4E0914407F0E079
:105A2000EE0FFF1FEB5EF84F0190F081E02DF7FFC6
:105A300003C0F095E195FF4F7A978CF08091660452
:105A40009091670462E070E00E94063DCB0162E045
:105A500070E00E94063D7093670460936604609155
:105A6000940770919507809196079091970720E091
:105A700031E040E050E00E943B3DC901DA018093F3
:105A8000940790939507A0939607B093970760911A
:105A90008C0770918D0780918E0790918F0720E081
:105AA00031E040E050E00E943B3DC901DA018093C3
:105AB0008C0790938D07A0938E07B0938F07E0908B
:105AC0000E04F0900F0400911004109111048091C5
:105AD0000A0490910B04A0910C04B0910D04E81AF3
:105AE000F90A0A0B1B0BE092B104F092B204009386
:105AF000B3041093B404209116043091170440911C
:105B00001804509119048091120490911304A091EB
:105B10001404B0911504281B390B4A0B5B0B20931E
:105B2000AD043093AE044093AF045093B004E092C0
:105B3000A904F092AA040093AB041093AC04209340
:105B4000A5043093A6044093A7045093A804809121
:105B50002E0490912F04A0913004B09131048E193D
:105B60009F09A00BB10B80932E0490932F04A09358
:105B70003004B09331048091360490913704A091A1
:105B80003804B0913904821B930BA40BB50B80939E
:105B9000360490933704A0933804B093390460918D
:105BA0001A0470911B0480911C0490911D042AE139
:105BB00030E040E050E00E943B3D3093DC06209313
:105BC000DB0660911E0470911F0480912004909167
:105BD00021042AE130E040E050E00E943B3D309358
:105BE000DE062093DD068091A9049091AA0490938B
:105BF000E0068093DF068091A5049091A60490931F
:105C0000E2068093E10660919C0770919D07809168
:105C10009E0790919F072AE130E040E050E00E940B
:105C20003B3D3093E4062093E3066091A00770911A
:105C3000A1078091A2079091A3072AE130E040E0FC
:105C400050E00E943B3D3093E6062093E5068091AC
:105C50009204909193049093F4068093F3068091BC
:105C60006404909165049C01B3E0220F331FBA9540
:105C7000E1F7880F991F280F391F3093F6062093FC
:105C8000F50681E090E090939104809390048091D8
:105C90009C0790919D07A0919E07B0919F0720912E
:105CA00088043091890440918A0450918B04281B08
:105CB000390B4A0B5B0B57FF07C050954095309549
:105CC00021953F4F4F4F5F4F20523E444040504040
:105CD0000CF0D7C02091A9043091AA044091AB04E4
:105CE0005091AC042130E0E13E07E0E04E07E0E0F7
:105CF0005E070CF453C080918F04882309F44AC0D6
:105D0000DA01C901FCE0B595A79597958795FA95B5
:105D1000D1F701969093910480939004CA01B90140
:105D200028E030E040E050E00E943B3DC901DA014C
:105D30008093960490939704A0939804B093990449
:105D400089589341A040B04064F088E893E1A0E016
:105D5000B0E08093960490939704A0939804B09336
:105D600099046091960470919704809198049091A1
:105D7000990420E031E040E050E00E943B3D8091FA
:105D8000660490916704820F931F90936704809339
:105D9000660406C081E080938F0402C010928F04D5
:105DA0004091A9045091AA046091AB047091AC0495
:105DB000403020EF52072FEF62072FEF72070CF0F1
:105DC0005DC080918E04882309F454C088279927E8
:105DD000DC01841B950BA60BB70BECE0B595A795E2
:105DE00097958795EA95D1F7209190043091910489
:105DF000280F391F3093910420939004CB01BA01EE
:105E000028E030E040E050E00E943B3DC901DA016B
:105E10008093960490939704A0939804B093990468
:105E200088579C4EAF4FBF4F64F488E79CEEAFEFAE
:105E3000BFEF8093960490939704A0939804B09337
:105E400099046091960470919704809198049091C0
:105E5000990420E031E040E050E00E943B3D809119
:105E6000660490916704820F931F90936704809358
:105E700066040BC081E080938E0407C010928E04EC
:105E800004C0109291041092900480916F07282F03
:105E900030E080919004909191042817390724F400
:105EA00030939104209390048091A9049091AA04C6
:105EB000A091AB04B091AC0481509440A040B0409C
:105EC00074F08091F6039091F70320919004309143
:105ED0009104820F931F9093F7038093F6038091B0
:105EE000A9049091AA04A091AB04B091AC04805095
:105EF0009C4FAF4FBF4F74F48091F6039091F7031E
:105F00002091900430919104821B930B9093F7039E
:105F10008093F60381E090E0909391048093900445
:105F2000109292041092930410929404109295048B
:105F30008091A0079091A107A091A207B091A3071B
:105F40002091840430918504409186045091870407
:105F5000281B390B4A0B5B0B57FF07C05095409528
:105F6000309521953F4F4F4F5F4F20523E44404068
:105F700050400CF0DDC0E090A504F090A604009124
:105F8000A7041091A80471E0E71670E1F70670E02D
:105F9000070770E017070CF458C080918D04882320
:105FA00009F44FC0A80197016CE0559547953795C6
:105FB00027956A95D1F78091900490919104820F72
:105FC000931F9093910480939004C801B70128E037
:105FD00030E040E050E00E943B3DC901DA0180938F
:105FE000920490939304A0939404B09395048958D9
:105FF0009341A040B04064F088E893E1A0E0B0E0B5
:106000008093920490939304A0939404B093950486
:1060100060919204709193048091940490919504FE
:1060200020E031E040E050E00E943B3D809164047C
:1060300090916504820F931F90936504809364048C
:1060400006C081E080938D0402C010928D044091BF
:10605000A5045091A6046091A7047091A804403053
:10606000F0EF5F07FFEF6F07FFEF7F070CF05DC0FA
:1060700080918C04882309F454C088279927DC0177
:10608000841B950BA60BB70B2CE0B595A7959795A0
:1060900087952A95D1F72091900430919104280F8B
:1060A000391F3093910420939004CB01BA0128E06A
:1060B00030E040E050E00E943B3DC901DA018093AE
:1060C000920490939304A0939404B09395048857FA
:1060D0009C4EAF4FBF4F64F488E79CEEAFEFBFEF2D
:1060E0008093920490939304A0939404B0939504A6
:1060F000609192047091930480919404909195041E
:1061000020E031E040E050E00E943B3D809164049B
:1061100090916504820F931F9093650480936404AB
:106120000BC081E080938C0407C010928C0404C0E3
:10613000109291041092900480916F07282F30E004
:1061400080919004909191042817390724F430939A
:106150009104209390048091A5049091A604A091AD
:10616000A704B091A80481509440A040B04074F0BE
:106170008091F8039091F90320919004309191045B
:10618000820F931F9093F9038093F8038091A504E5
:106190009091A604A091A704B091A80480509C4FB0
:1061A000AF4FBF4F74F48091F8039091F9032091A1
:1061B000900430919104821B930B9093F903809388
:1061C000F80380919204909193049093F006809349
:1061D000EF068091F6039091F7039093E806809381
:1061E000E7068091F8039091F9032091FC03309128
:1061F000FD03821B930B9C0103E0220F331F0A95C2
:10620000E1F7880F991F280F391F3093EA06209372
:10621000E90608C0109265041092640410926704A5
:106220001092660420E030E040E050E06091A40766
:106230007091A5078091A6079091A7070E94113B36
:10624000882341F41092650410926404109267044C
:106250001092660480919C0790919D07A0919E07E3
:10626000B0919F078093880490938904A0938A0437
:10627000B0938B048091A0079091A107A091A207F1
:10628000B091A3078093840490938504A09386041F
:10629000B093870410921A0410921B0410921C04ED
:1062A00010921D0410921E0410921F0410922004DC
:1062B00010922104109222041092230410922404BC
:1062C0001092250410929C0710929D0710929E0731
:1062D00010929F071092A0071092A1071092A20798
:1062E0001092A307109294071092950710929607A8
:1062F0001092970710928C0710928D0710928E07BC
:1063000010928F071092E1031092E00380915B04DA
:1063100090915C0497FF03C0909581959F4F45979E
:106320003CF08091490784FD03C081E080939A048A
:10633000F0905207C0905B04D0905C04B6018827AF
:1063400077FD8095982F2F2D30E040E050E00E949F
:10635000C73CF601D7FE04C0EE27FF27EC19FD0964
:106360009F01442737FD4095542F0E94C73C20E0F1
:1063700032E040E050E00E943B3D89019A018F2DC0
:1063800090E0BC016C9DC0016D9D900D7C9D900DB9
:10639000112464E070E00E94063D600F711F8827A1
:1063A00077FD8095982F6093B5047093B604809321
:1063B000B7049093B80420913A0430913B04409183
:1063C0003C0450913D04261B370B480B590B20937E
:1063D0003A0430933B0440933C0450933D04809135
:1063E0003A0490913B04A0913C04B0913D04815546
:1063F000934CA040B04064F080E593ECA0E0B0E0A6
:1064000080933A0490933B04A0933C04B0933D04E2
:1064100080913A0490913B04A0913C04B0913D04DA
:10642000805B9C43AF4FBF4F64F480EB9CE3AFEFC6
:10643000BFEF80933A0490933B04A0933C04B09345
:106440003D048091460490914704892B09F498C03B
:106450008091490783FF94C060910A0470910B04F6
:1064600080910C0490910D0420E032E040E050E077
:106470000E943B3D890137FF03C0109501951F4FD6
:10648000609112047091130480911404909115048A
:1064900020E032E040E050E00E943B3DA90137FFA0
:1064A00003C0509541955F4F401751070CF4A80168
:1064B00049315105A4F480919A04882381F0809198
:1064C000820490918304892B51F480914604909129
:1064D0004704909349048093480410929A042091B1
:1064E000980330E0429FC001439F900D529F900D52
:1064F0001124B6E095958795BA95E1F7A901481B57
:10650000590B14161506B4F58091820490918304FA
:10651000892B41F500913A0410913B0420913C04F1
:1065200030913D0480914A0490914B04BC01469FF8
:10653000C001479F900D569F900D112460E270E0BE
:106540000E94063D882777FD8095982F600F711F68
:10655000821F931F60933A0470933B0480933C0422
:1065600090933D048091820490918304009741F0C0
:10657000019702C084EF91E090938304809382049A
:1065800080919B04815080939B048F5F09F078C0B9
:1065900088E180939B0460910A0470910B048091C0
:1065A0000C0490910D04E0905507FF2400E010E0EA
:1065B000A80197010E943B3D3093BA062093B9068B
:1065C0006091120470911304809114049091150449
:1065D000A80197010E943B3D3093BC062093BB0667
:1065E0008091AD079091AE079093BE068093BD0653
:1065F0008091B7079091B8079093C0068093BF062B
:106600008091B0079091B1079093C2068093C10624
:1066100080916004909161049093C4068093C306B6
:106620006091420470914304809144049091450428
:1066300020E032E040E050E00E943B3D3093C6064F
:106640002093C50680914604909147049093CA0612
:106650008093C9068091090390910A039093CC0618
:106660008093CB06809156048093CD061092CE067F
:1066700080919807909199079093DA068093D906B4
:10668000809168048823A9F0609191077091920726
:10669000882777FD8095982F0E94B03B2091B20704
:1066A0003091B3074091B4075091B5070E94643C04
:1066B00032C060910A0470910B0480910C04909197
:1066C0000D04E0909107F09092070E94B03B20915A
:1066D000A4073091A5074091A6075091A7070E94F3
:1066E000643C5B016C010027F7FC0095102FC8018A
:1066F000B7010E94B03B2091B2073091B30740919F
:10670000B4075091B5070E94643C9B01AC01C601DF
:10671000B5010E94AD3A0E947D3B70939207609351
:106720009107809169048823A9F06091890770918D
:106730008A07882777FD8095982F0E94B03B20918B
:10674000B2073091B3074091B4075091B5070E944A
:10675000643C32C06091120470911304809114045F
:1067600090911504E0908907F0908A070E94B03B51
:106770002091A4073091A5074091A6075091A70743
:106780000E94643C5B016C010027F7FC0095102F10
:10679000C801B7010E94B03B2091B2073091B30706
:1067A0004091B4075091B5070E94643C9B01AC0135
:1067B000C601B5010E94AD3A0E947D3B70938A07E5
:1067C000609389076091B0077091B107A09026048B
:1067D000B0902704C0902804D0902904882777FD22
:1067E0008095982F0E94B03B7B018C016091B2078D
:1067F0007091B3078091B4079091B5079B01AC01EC
:106800000E94AD3A9B01AC01C801B7010E94643CF3
:106810007B018C01C601B5010E94B03B2091A40709
:106820003091A5074091A6075091A7070E94643CAC
:1068300020E030E040E05FE30E94643C9B01AC015B
:10684000C801B7010E94AD3A0E947D3B7093B10729
:106850006093B00760911204709113048091140446
:10686000909115040E94B03B2091A4073091A50798
:106870004091A6075091A7070E94643C0E94823B6A
:106880007093EC066093EB068091590490915A0442
:106890009093F8068093F7068091890790918A0774
:1068A0009093F2068093F106809191079091920760
:1068B0008150984034F080E098E090939207809364
:1068C000910780919107909192078050984F34F4EE
:1068D00080E098EF909392078093910780918907C9
:1068E00090918A078150984034F080E098E090932E
:1068F0008A07809389078091890790918A07805041
:10690000984F34F480E098EF90938A07809389073A
:106910008091B0079091B1078150984034F080E0A9
:1069200098E09093B1078093B0078091B007909161
:10693000B1078050984F34F480E098EF9093B107FE
:106940008093B0078091490780FFDFC09091950345
:1069500081FF0EC0923310F5809160049091610424
:106960004497909363048093620410924D0419C07D
:106970002091A0033091A103290F311D80914E0772
:1069800090E0AC01249FC001259F900D349F900D95
:1069900011244497909363048093620481E0809370
:1069A0004D0480914C04882321F0109263041092CE
:1069B000620420916004309161044091620450911E
:1069C0006304421753070CF0A0C080914D04882344
:1069D00009F49BC08091960390E0241B350BBC0109
:1069E000629FC001639F900D729F900D112460E122
:1069F00070E00E94063D5B01C090DE03D090DF0393
:106A00006091420470914304809144049091450444
:106A1000E0909703FF2400E010E020E032E040E047
:106A200050E00E943B3DC801B7010E94C73C20E2F4
:106A300030E040E050E00E943B3DF9017FEF2E3C0A
:106A4000370714F4EEECFFEF8091940390E0DC0143
:106A5000AC9DC001AD9D900DBC9D900D112468E0D2
:106A600070E00E94063D80919C0490919D049C01E1
:106A7000A4E0220F331FAA95E1F7281B390B261B30
:106A8000370B2A193B09CF01E333F10514F082E3F8
:106A900090E0281B390B89819A81820F931F60E156
:106AA00070E00E94063D70939D0460939C042091C9
:106AB0004A0730E062177307ACF4E981FA81E21704
:106AC000F30724F030939D0420939C0480914A079F
:106AD00090E029813A812817390724F430939D04E6
:106AE00020939C0480919C0490919D0449815A813B
:106AF0004817590724F450939D0440939C046091D7
:106B00009C0470919D047A8369838091AF07282F3C
:106B100030E0C9014397A981BA81A817B90724F0C9
:106B2000F9017497FA83E98329813A813093C80681
:106B30002093C7062091B0073091B1078091B5042A
:106B40009091B604A091B704B091B8044091AF07FA
:106B500069817A81643171051CF4222433242EC0AA
:106B6000E42FF0E0A901481B590BCA0129813A81A1
:106B700035952795821793070CF49C0189819A819A
:106B800062E070E00E94063D709561957F4FC901FB
:106B9000261737070CF4CB019F0169817A81261BE8
:106BA000370B281739070CF4C90129813A812E1BAC
:106BB0003F0B1C01821793070CF419018091910778
:106BC000909192074090C9045090CA04840D951D7D
:106BD000A0915704B0915804B887AF838A1B9B0BD0
:106BE00090939B0780939A076090A4077090A507E5
:106BF0008090A6079090A70720E030E040E050E0AA
:106C0000C401B3010E94113B882309F440C0E09005
:106C10000A04F0900B0400910C0410910D04609193
:106C2000BD047091BE048091BF049091C0040E9485
:106C3000B03B5B016C01C801B7010E94B03BA401ED
:106C400093010E94643C7B018C01EF81F885E4197B
:106C5000F509BF01882777FD8095982F0E94B03BEA
:106C60009B01AC01C801B7010E94AC3A9B01AC0189
:106C7000C601B5010E94AD3A0E947D3B6093BD0400
:106C80007093BE048093BF049093C0041CC02091F5
:106C90009A0730919B07442737FD4095542F8091E8
:106CA000BD049091BE04A091BF04B091C004820FB6
:106CB000931FA41FB51F8093BD049093BE04A0939F
:106CC000BF04B093C0048091BD049091BE04A09114
:106CD000BF04B091C00481589E43A040B04064F00E
:106CE00080E89EE3A0E0B0E08093BD049093BE04F2
:106CF000A093BF04B093C0048091BD049091BE04E2
:106D0000A091BF04B091C0048058914CAF4FBF4FC9
:106D100064F480E891ECAFEFBFEF8093BD049093F3
:106D2000BE04A093BF04B093C00460919A07709111
:106D30009B07882777FD8095982F0E94B03B7B01A9
:106D40008C016091BD047091BE048091BF0490914C
:106D5000C0040E94B03B2091900330919103409178
:106D60009203509193030E94643C9B01AC01C801C3
:106D7000B7010E94AD3A0E947D3B8B01C10137FEF5
:106D800004C0882799278219930995958795498189
:106D90005A81840F951F9C01442737FD4095542F3D
:106DA0002B833C834D835E8320919F0330E040E042
:106DB00050E06B817C818D819E810E94C73C20E4E4
:106DC00030E040E050E00E943B3DA901622F232FBC
:106DD000041715071CF4C801602F292FEE27FF2781
:106DE000E41BF50B862F922FBC016E177F070CF466
:106DF000BF01E981FA81E20DF31D9F01260F371FC4
:106E000037FF03C020E030E008C08091AF07482F73
:106E100050E0421753070CF49A0180919307482FD2
:106E200050E0241735070CF49A0120938B079F013B
:106E3000261B370B37FF03C020E030E008C08091ED
:106E4000AF07482F50E0421753070CF49A01809186
:106E50009307482F50E0C901241735070CF4CA01E5
:106E6000809390078091890790918A074090CB0486
:106E70005090CC04840D951D4091590450915A04B2
:106E800058874F83841B950B9093880780938707BF
:106E90006090A4077090A5078090A6079090A70720
:106EA00020E030E040E050E0C401B3010E94113B1B
:106EB000882309F441C0E0901204F090130400917B
:106EC0001404109115046091B9047091BA04809172
:106ED000BB049091BC040E94B03B5B016C01C801F3
:106EE000B7010E94B03BA40193010E94643C7B0166
:106EF0008C016F81788564197509DB01BD018827D4
:106F000077FD8095982F0E94B03B9B01AC01C80192
:106F1000B7010E94AC3A9B01AC01C601B5010E94C9
:106F2000AD3A0E947D3B6093B9047093BA0480939C
:106F3000BB049093BC041CC0209187073091880744
:106F4000442737FD4095542F8091B9049091BA049D
:106F5000A091BB04B091BC04820F931FA41FB51F66
:106F60008093B9049093BA04A093BB04B093BC047B
:106F70008091B9049091BA04A091BB04B091BC0473
:106F800081589E43A040B04064F080E89EE3A0E0BA
:106F9000B0E08093B9049093BA04A093BB04B0937B
:106FA000BC048091B9049091BA04A091BB04B09143
:106FB000BC048058914CAF4FBF4F64F480E891EC13
:106FC000AFEFBFEF8093B9049093BA04A093BB04D2
:106FD000B093BC046091870770918807882777FD7C
:106FE0008095982F0E94B03B7B018C016091B90481
:106FF0007091BA048091BB049091BC040E94B03B94
:10700000209190033091910340919203509193030A
:107010000E94643C9B01AC01C801B7010E94AD3ADB
:107020000E947D3B7B018C0120919F0330E040E07A
:1070300050E06B817C818D819E810E94C73C20E461
:1070400030E040E050E00E943B3DC901422F232F39
:10705000E816F90614F44E2D2F2D66277727681BA6
:10706000790B842F922F9C01261737070CF49B0174
:1070700049815A8142195309420F531F57FF03C0D8
:1070800040E050E008C08091AF07682F70E06417BF
:1070900075070CF4AB0180919307682F70E04617D9
:1070A00057070CF4AB014093AA0749815A81421B50
:1070B000530B9A012219330937FF03C020E030E057
:1070C00007C08091AF0790E0821793070CF49C01F2
:1070D0008091930790E0281739070CF49C012093C6
:1070E000A80728960FB6F894DEBF0FBECDBFCF918C
:1070F000DF911F910F91FF90EF90DF90CF90BF90A5
:10710000AF909F908F907F906F905F904F903F9047
:107110002F90089581E08093410722E02093420759
:1071200083E08093430754E05093440745E0409345
:10713000450736E03093460787E08093470788E0AD
:107140008093480780EC809349079EE190934A071B
:107150008BEF80934C078AE080934D0790934B0709
:1071600090934F0720934E07209350075093510759
:10717000309352078FE0809353078AEF8093540730
:107180009093550780E88093560724E6209357078D
:107190008CE8809358078EE58093590783E28093AB
:1071A0005A0784E180935B0710925C0780E180932B
:1071B0005D0780E580935E0710925F07109260077D
:1071C0001092610710927107109272071092730764
:1071D000109274072093620788E2809363071092ED
:1071E000760792E39093640786E98093650740935E
:1071F0006607909367078AE580936807909369070D
:107200001092750780936A0740936B0720936C0771
:1072100020936D0780E280936E0750936F079093E1
:107220007007ABE7B7E0EDE6F3E08CE001900D927C
:107230008150E1F7089581E08093410782E08093D7
:10724000420723E02093430754E05093440745E06E
:107250004093450736E03093460787E08093470721
:1072600088E08093480780E4809349079EE19093EB
:107270004A078BEF80934C078AE080934D079093E9
:107280004B0790934F0720934E072093500750933E
:107290005107309352078FE0809353078AEF809312
:1072A00054079093550780E88093560790E5909394
:1072B000570788E7809358078EE58093590783E244
:1072C00080935A0784E180935B0710925C0730E259
:1072D00030935D0790935E0710925F0710926007EE
:1072E0001092610710927107109272071092730743
:1072F0001092740724E62093620788E28093630764
:107300001092760792E39093640786E9809365076D
:1073100040936607909367078AE580936807909388
:1073200069071092750780936A0740936B07209353
:107330006C0720936D0730936E0750936F078BE4B3
:1073400080937007ABE7B7E0E7E7F3E08CE00190EC
:107350000D928150E1F7089581E08093410782E02A
:107360008093420783E08093430734E030934407DF
:1073700045E04093450786E08093460787E0809389
:10738000470728E02093480780E4809349079EE15F
:1073900090934A078BEF80934C078AE080934D07C8
:1073A00090934B0790934F0730934E0730935007BD
:1073B000209351078CE0809352078FE0809353070E
:1073C0008AEF809354079093550790E8909356075F
:1073D00080E58093570756E9509358078EE58093D0
:1073E000590783E280935A0784E180935B071092E8
:1073F0005C0780E280935D0790935E0710925F07C1
:107400001092600710926107109271071092720734
:10741000109273071092740724E62093620788E2A3
:10742000809363071092760782E3809364075093FA
:10743000650740936607809367079AE5909368070E
:10744000809369071092750790936A0740936B07C2
:1074500020936C0720936D0780E180936E07309333
:107460006F0720937007ABE7B7E0EFE7F3E08CE03E
:1074700001900D928150E1F708958091CD04909193
:10748000CE04A091CF04B091D0048093D504909302
:10749000D604A093D704B093D8048091D1049091DE
:1074A000D204A091D304B091D4048093D9049093D2
:1074B000DA04A093DB04B093DC0408951092CA04AC
:1074C0001092C9041092CC041092CB040895FC01D0
:1074D0004150504030F001900616D1F73197CF015E
:1074E0000895882799270895A0E0B0E0EAE7FAE335
:1074F0000C94603D7C01EB018A01690109C0CE0159
:107500002196F6010995F70181937F010150104002
:1075100001151105A1F7CDB7DEB7E8E00C947C3D6D
:10752000A0E0B0E0E6E9FAE30C94603DEC017B01F9
:107530008A01690109C0F70161917F01CE0121969D
:10754000F60109950150104001151105A1F7CDB7BD
:10755000DEB7E8E00C947C3D5058BB27AA270ED03C
:1075600075C166D130F06BD120F031F49F3F11F43A
:107570001EF45BC10EF4E095E7FB51C1E92F77D112
:1075800080F3BA17620773078407950718F071F440
:107590009EF58FC10EF4E0950B2EBA2FA02D0B0196
:1075A000B90190010C01CA01A0011124FF27591B48
:1075B00099F0593F50F4503E68F11A16F040A22F4E
:1075C000232F342F4427585FF3CF469537952795BF
:1075D000A795F0405395C9F77EF41F16BA0B620BBE
:1075E000730B840BBAF09150A1F0FF0FBB1F661F05
:1075F000771F881FC2F70EC0BA0F621F731F841F48
:1076000048F4879577956795B795F7959E3F08F06D
:10761000B3CF9395880F08F09927EE0F979587952C
:107620000895D9D008F481E008950CD00FC107D196
:1076300040F0FED030F021F45F3F19F0F0C051115E
:1076400039C1F3C014D198F39923C9F35523B1F389
:10765000951B550BBB27AA2762177307840738F0C1
:107660009F5F5F4F220F331F441FAA1FA9F333D020
:107670000E2E3AF0E0E830D091505040E695001CD4
:10768000CAF729D0FE2F27D0660F771F881FBB1F90
:10769000261737074807AB07B0E809F0BB0B802D6A
:1076A000BF01FF2793585F4F2AF09E3F510568F0B6
:1076B000B6C000C15F3FECF3983EDCF3869577954A
:1076C0006795B795F7959F5FC9F7880F911D9695B8
:1076D000879597F90895E1E0660F771F881FBB1F14
:1076E000621773078407BA0720F0621B730B840BC1
:1076F000BA0BEE1F88F7E095089504D06894B11195
:10770000D9C00895BCD088F09F5790F0B92F992721
:10771000B751A0F0D1F0660F771F881F991F1AF09C
:10772000BA95C9F712C0B13081F0C3D0B1E0089565
:10773000C0C0672F782F8827B85F39F0B93FCCF3E6
:10774000869577956795B395D9F73EF49095809592
:10775000709561957F4F8F4F9F4F0895E89409C0B2
:1077600097FB3EF490958095709561957F4F8F4F74
:107770009F4F9923A9F0F92F96E9BB279395F6958A
:10778000879577956795B795F111F8CFFAF4BB0F08
:1077900011F460FF1BC06F5F7F4F8F4F9F4F16C06C
:1077A000882311F096E911C0772321F09EE8872FF6
:1077B000762F05C0662371F096E8862F70E060E0B2
:1077C0002AF09A95660F771F881FDAF7880F96952B
:1077D000879597F90895990F0008550FAA0BE0E8CF
:1077E000FEEF16161706E807F907C0F01216130683
:1077F000E407F50798F0621B730B840B950B39F4C3
:107800000A2661F0232B242B252B21F408950A2628
:1078100009F4A140A6958FEF811D811D089597F968
:107820009F6780E870E060E008959FEF80EC089526
:1078300000240A941616170618060906089500244F
:107840000A9412161306140605060895092E0394C9
:10785000000C11F4882352F0BB0F40F4BF2B11F43D
:1078600060FF04C06F5F7F4F8F4F9F4F089557FD9C
:107870009058440F551F59F05F3F71F04795880F9E
:1078800097FB991F61F09F3F79F087950895121635
:1078900013061406551FF2CF4695F1DF08C01616E1
:1078A00017061806991FF1CF869571056105089492
:1078B0000895E894BB2766277727CB0197F90895A9
:1078C0008ADF08F48FEF08950BD0C0CFB1DF28F026
:1078D000B6DF18F0952309F0A2CFA7CF1124EACF85
:1078E000C6DFA0F3959FD1F3950F50E0551F629F1F
:1078F000F001729FBB27F00DB11D639FAA27F00D09
:10790000B11DAA1F649F6627B00DA11D661F829F2F
:107910002227B00DA11D621F739FB00DA11D621F14
:10792000839FA00D611D221F749F3327A00D611D31
:10793000231F849F600D211D822F762F6A2F112413
:107940009F5750408AF0E1F088234AF0EE0FFF1F66
:10795000BB1F661F771F881F91505040A9F79E3F9D
:10796000510570F05CCFA6CF5F3FECF3983EDCF39F
:10797000869577956795B795F795E7959F5FC1F7DA
:10798000FE2B880F911D9695879597F90895629F14
:10799000D001739FF001829FE00DF11D649FE00D07
:1079A000F11D929FF00D839FF00D749FF00D659F68
:1079B000F00D9927729FB00DE11DF91F639FB00D67
:1079C000E11DF91FBD01CF0111240895991B79E034
:1079D00004C0991F961708F0961B881F7A95C9F75F
:1079E00080950895AA1BBB1B51E107C0AA1FBB1FAE
:1079F000A617B70710F0A61BB70B881F991F5A953B
:107A0000A9F780959095BC01CD01089597FB092EAB
:107A100007260AD077FD04D0E5DF06D000201AF44F
:107A2000709561957F4F0895F6F7909581959F4FDA
:107A30000895A1E21A2EAA1BBB1BFD010DC0AA1FAF
:107A4000BB1FEE1FFF1FA217B307E407F50720F0C7
:107A5000A21BB30BE40BF50B661F771F881F991F42
:107A60001A9469F760957095809590959B01AC018B
:107A7000BD01CF01089597FB092E05260ED057FDB5
:107A800004D0D7DF0AD0001C38F4509540953095CB
:107A900021953F4F4F4F5F4F0895F6F79095809592
:107AA000709561957F4F8F4F9F4F08952F923F9212
:107AB0004F925F926F927F928F929F92AF92BF92FE
:107AC000CF92DF92EF92FF920F931F93CF93DF93AA
:107AD000CDB7DEB7CA1BDB0B0FB6F894DEBF0FBE07
:107AE000CDBF09942A88398848885F846E847D8454
:107AF0008C849B84AA84B984C884DF80EE80FD8056
:107B00000C811B81AA81B981CE0FD11D0FB6F894CB
:0E7B1000DEBF0FBECDBFED010895F894FFCF8C
:107B1E000A01FF64496E74656772616C4E69636B2E
:107B2E0020202020496E74656772616C526F6C6CF8
:107B3E00202020204163634E69636B20202020208B
:107B4E0020202020416363526F6C6C202020202067
:107B5E00202020204779726F4769657220202020EF
:107B6E0020202020486F6568656E5765727420204E
:107B7E00202020204163635A202020202020202016
:107B8E00202020204761732020202020202020202C
:107B9E00202020204B6F6D7061737356616C75657C
:107BAE00202020205370616E6E756E67202020207D
:107BBE0020202020456D7066616E672020202020D9
:107BCE0020202020416E616C6F67313120202020F3
:107BDE00202020204D6F746F725F566F726E65207D
:107BEE00202020204D6F746F725F48696E74656E31
:107BFE00202020204D6F746F725F4C696E6B732066
:107C0E00202020204D6F746F725F5265636874730D
:107C1E00202020204163635F5A2020202020202036
:107C2E00202020204D697474656C4163634E696336
:107C3E006B2020204D697474656C416363526F6CC8
:107C4E006C202020496E74656772616C4572724EAD
:107C5E0069636B20496E74656772616C457272520E
:107C6E006F6C6C204D697474656C496E744E6963EB
:107C7E006B2020204D697474656C496E74526F6C64
:107C8E006C0920004E65757472616C4E69636B20D1
:107C9E0020202020526F6C6C4F6666736574202016
:107CAE0020202020496E74526F6C6C2A46616B74D2
:107CBE006F722020416E616C6F673236202020205B
:107CCE0020202020446972656B74417573676C5275
:107CDE006F6C6C204D65737377657274526F6C6C3C
:107CEE0020202020417573676C65696368526F6C44
:107CFE006C202020492D4C616765526F6C6C2020E2
:107D0E0020202020537469636B526F6C6C202020EE
:107D1E0020202020FFFF010A016400007D0000FFEB
:107D2E00030102030405060708090A48616C6C6F1B
:107D3E002057656C74000000000000000000000079
:107D4E000000000000000000000000000000000025
:107D5E000000000000000000000000000000000015
:107D6E000000000000000000000000000000000005
:107D7E0000000000000000000000000B01426567DB
:107D8E00696E6E657200004E6F726D616C0000530D
:107D9E00706F72740000640090D0030090D00300E6
:107DAE0017B7D13830FB103A409696020A644664F3
:047DBE00ECFFC0070F
:00000001FF
